:020000040800F2
:1000000000C00120FD7B0008497C0008497C0008F5
:10001000497C0008497C0008497C00080000000079
:10002000000000000000000000000000497C000803
:10003000497C000800000000497C00089519000870
:10004000497C0008497C0008497C0008497C00087C
:10005000497C0008497C0008497C0008497C00086C
:10006000497C0008B5190008497C0008497C000853
:10007000497C0008497C0008497C0008497C00084C
:10008000497C0008497C0008497C0008497C00083C
:10009000497C0008497C0008497C0008497C00082C
:1000A000497C0008497C0008497C0008497C00081C
:1000B000497C0008497C0008497C0008497C00080C
:1000C000497C0008497C0008497C0008C9190008DF
:1000D000497C0008497C0008497C0008497C0008EC
:1000E000497C0008497C0008497C0008497C0008DC
:1000F000497C0008497C0008497C0008497C0008CC
:10010000497C0008497C0008497C0008497C0008BB
:10011000497C0008497C0008497C0008497C0008AB
:10012000497C0008497C0008497C0008497C00089B
:10013000497C00080000000000000000497C000825
:10014000497C0008497C0008497C0008A519000882
:10015000497C0008497C0008497C0008497C00086B
:10016000497C0008497C0008497C0008497C00085B
:10017000497C0008497C00080000000000000000E5
:10018000497C0008497C000880B483B000AF034676
:100190003960FB713B6812221A80034B18460C37FA
:1001A000BD465DF8047B70471C00002080B483B01E
:1001B00000AF03463960FB713B6804221A80034B91
:1001C00018460C37BD465DF8047B704730000020B0
:1001D00080B582B000AF03463960FB710448054921
:1001E0003A6802F0D5F8034B18460837BD4680BD83
:1001F000007E00087401002080B582B000AF034685
:100200003960FB71044805493A6802F0C1F8034BB4
:1002100018460837BD4680BD147E000874010020D2
:1002200080B582B000AF03463960FB7104480549D0
:100230003A6802F0ADF8034B18460837BD4680BD5A
:10024000287E00087401002080B582B000AF03460C
:100250003960FB71044805493A6802F099F8034B8C
:1002600018460837BD4680BD387E0008740100205E
:1002700080B582B000AF03463960FB710448054980
:100280003A6802F085F8034B18460837BD4680BD32
:10029000447E00087401002080B588B000AF78600B
:1002A0007B681B68B3F1A04F24D1144A134B5B6BDE
:1002B00043F080035363114A104B5B6C43F480435B
:1002C00053644FF4C053FB6002233B6100237B6106
:1002D0000023BB610A23FB6107F10C0308481946A0
:1002E00007F03EF943200A21002207F09FFB43203C
:1002F00007F0B8FB2037BD4680BD00BF0038024084
:100300000000024080B582B000AF78607B68D3F80F
:10031000B0237B6803F560731046194602F038F984
:100320000837BD4680BD00BF80B582B000AF7860A1
:100330000B46FB707B68D3F8B003FA7879681346F4
:10034000DB009B1A9B000B4403F5F0735B68FA78A3
:1003500011461A4602F066F90837BD4680BD00BF57
:1003600080B582B000AF78600B46FB707B68D3F835
:10037000B003FA7879681346DB009B1A9B000B44A4
:1003800038339B68FA7811461A4602F0A7F9083705
:10039000BD4680BD80B582B000AF78607B68D3F881
:1003A000B033184602F092FA0837BD4680BD00BF50
:1003B00080B584B000AF78600123FB737B68DB6895
:1003C000002B02D0022B03D005E00023FB7305E0D5
:1003D0000123FB7302E00123FB7300BF7B68D3F8AA
:1003E000B023FB7B1046194602F038FA7B68D3F83D
:1003F000B033184602F002FA1037BD4680BD00BF88
:1004000080B582B000AF78607B68D3F8B03318460F
:1004100002F034FA7B681B6803F560631A467B6858
:100420001B6803F560631B6843F001031360083722
:10043000BD4680BD80B582B000AF78607B681B6828
:1004400003F560631A467B681B6803F560631B68ED
:1004500023F0010313607B68D3F8B033184602F031
:1004600023FA0837BD4680BD80B582B000AF786002
:100470000B46FB707B68D3F8B023FB781046194617
:1004800002F04CFA0837BD4680BD00BF80B582B08F
:1004900000AF78600B46FB707B68D3F8B023FB7825
:1004A0001046194602F02CFA0837BD4680BD00BF41
:1004B00080B582B000AF78607B68D3F8B03318465F
:1004C00002F03AFA0837BD4680BD00BF80B582B061
:1004D00000AF78607B68D3F8B033184602F038FA82
:1004E0000837BD4680BD00BF80B582B000AF7860E0
:1004F0007B68D3F8B033184602F042FA0837BD469D
:1005000080BD00BF80B582B000AF78607B681B788B
:10051000002B3AD11F4A7B68C2F8B0337B681D4A72
:10052000C3F820221B4B4FF0A0421A60194B072240
:100530005A60184B0222DA60164B00221A61154BE2
:1005400000225A61134B02229A61124B0022DA6197
:10055000104B00221A620F4B00229A620D4B0022B0
:10056000DA620C4B00221A630A4805F0EFFF0948D3
:10057000802105F0D9FF07480021402205F086FFC1
:1005800004480121802205F081FF00231846083726
:10059000BD4680BD7403002080B582B000AF786096
:1005A0007B68D3F82032184606F0D8F800231846A6
:1005B0000837BD4680BD00BF80B582B000AF78600F
:1005C0007B68D3F82032184606F0EAF80023184674
:1005D0000837BD4680BD00BF80B582B000AF7860EF
:1005E000084611461A460346FB700B46BB7013467D
:1005F0003B807B68D3F82002F9783A88BB7806F014
:10060000CBFC002318460837BD4680BD80B582B0BC
:1006100000AF78600B46FB707B68D3F82022FB7834
:100620001046194606F020FD002318460837BD463F
:1006300080BD00BF80B582B000AF78600B46FB7014
:100640007B68D3F82022FB781046194606F0CEFED0
:10065000002318460837BD4680BD00BF80B582B074
:1006600000AF78600B46FB707B68D3F82022FB78E4
:100670001046194606F014FE002318460837BD46FA
:1006800080BD00BF80B582B000AF78600B46FB70C4
:100690007B68D3F82022FB781046194606F05CFEF2
:1006A000002318460837BD4680BD00BF80B485B022
:1006B00000AF78600B46FB707B68D3F82032FB609C
:1006C000FB785BB2002B0BDAFB7803F07F02F96852
:1006D0001346DB009B1A9B000B4430339B790BE0E5
:1006E000FB7803F07F02F9681346DB009B1A9B003E
:1006F0000B4403F5EC739B7818461437BD465DF840
:10070000047B704780B582B000AF78600B46FB7009
:100710007B68D3F82022FB781046194606F01AFCB5
:10072000002318460837BD4680BD00BF80B584B0A1
:1007300000AFF8607A601A460B46FB7213463B81A5
:10074000FB68D3F820123B89FA7A084611467A688A
:1007500006F04AFD002318461037BD4680BD00BF95
:1007600080B584B000AFF8607A601A460B46FB7221
:1007700013463B81FB68D3F820123B89FA7A08467E
:1007800011467A6806F0BAFC002318461037BD46B9
:1007900080BD00BF80B582B000AF78600B46FB70B3
:1007A0007B68D3F82022FB781046194606F002FD3C
:1007B000034618460837BD4680BD00BF80B500AF70
:1007C00002480349002201F03DFE80BD28070020B9
:1007D0000000002080B582B000AF00F04BF900F0BF
:1007E000D3F938603B68002B03D1174B03221A70F2
:1007F00026E03B6840F201129A803B6800229A7121
:100800003B680022DA71FF237B710023FB800AE042
:10081000FB883A6813447A791A727B7927337B71A3
:10082000FB880133FB80FB88B3F5007FF0D3386889
:1008300000F006FA0346002B02D1044800F08EFBBC
:100840000837BD4680BD00BF48010020B108000840
:1008500080B500AF074B03221A70074B1B78002BA3
:1008600006D0054B1B78012B02D8044801F03AFE54
:1008700080BD00BF4801002049010020280700205A
:1008800080B500AF094B1B78032B01D101230AE08F
:10089000064B1B78022B05D0642001F029F8FFF7E6
:1008A000D7FFFEE70023184680BD00BF48010020A7
:1008B00080B584B000AF78601F4B1B78022B00D945
:1008C00037E01D4B1B78002B02D17B68002B05D134
:1008D000642001F00DF8FFF7BBFFFEE77B689B8803
:1008E00040F20112934205D0642001F001F8FFF7B5
:1008F000AFFFFEE7FF237B730023FB8112E0FB8940
:100900007A6813441B7A7A7B9A4205D0642000F0FF
:10091000EFFFFFF79DFFFEE77B7B27337B73FB89B0
:100920000133FB81FB89B3F5007FE8D3786800F0E1
:1009300005F81037BD4680BD4801002080B582B063
:1009400000AF78600B4B01221A707B6801229A80FD
:100950007B6800229A717B680122DA71786800F066
:100960006FF90346002B02D1034800F0F7FA08376D
:10097000BD4680BD480100207D09000880B584B0D7
:1009800000AF78600023FB73274B1B78022B00D944
:1009900047E0254B1B78012B02D17B68002B05D14A
:1009A000642000F0A5FFFFF753FFFEE77B689B88FC
:1009B000022B05D0642000F09BFFFFF749FFFEE704
:1009C0007B681B7A012B04D10123FB73174BBB609F
:1009D00000BF786800F000F9FB7B002B05D1642094
:1009E00000F086FFFFF734FFFEE7114B1B78002B6A
:1009F0000AD00F4B1B78FA7B9A4205D0642000F096
:100A000077FFFFF725FFFEE7074B02221A70084A1F
:100A1000FB7B13700748B96801F03EFD054801F003
:100A200055FD1037BD4680BD480100203400002030
:100A3000490100202807002080B500AF0A4B1B7831
:100A4000002B03D0084B1B78012B05D9642000F044
:100A50004FFFFFF7FDFEFEE7044801F043FD0448A9
:100A600000F056F880BD00BF490100202807002093
:100A70003D09000880B500AF1F4B00221A701F4BC4
:100A800000221A701E4B1F4A1A601D4B002283F869
:100A900051201B4B4FF482725A60194B00229A600E
:100AA000174B4FF40062DA60154B00221A61144BA9
:100AB00000225A61124B4FF400729A61104B2022AF
:100AC000DA610F4B00221A620D4B00225A620C4B66
:100AD0004FF400529A620A4B0722DA62084804F087
:100AE000F3FC094B1B6903F00803002B02D1074BF1
:100AF00001221A7080BD00BF600B00205409002045
:100B00006C0D002000300140000002405C0100201C
:100B100080B582B000AF7860174B1B78082B01D9E5
:100B2000012325E0154B1B68002B05D0642000F045
:100B3000DFFEFFF78DFEFEE7114B1B78002B07D180
:100B40000F4B01221A707B680D48984700230FE075
:100B50000C4B1B78002B07D10A4B01221A707B68C3
:100B600008489847002303E0044A7B681360002389
:100B700018460837BD4680BD5001002054010020B2
:100B8000600B00205409002080B500AF0F4B1B788C
:100B9000082B01D9002317E00D4B1B78002B04D143
:100BA0000B4B01221A700A4B0EE00A4B1B78002BEC
:100BB00004D1084B01221A70064B05E0642000F0B6
:100BC00097FEFFF745FEFEE7184680BD5001002066
:100BD000600B00205409002080B584B000AF78601D
:100BE000134B1B78082B00D91EE07B68114A9342F7
:100BF00009D07B68104A934205D0642000F078FE4B
:100C0000FFF726FEFEE70D4B1B68002B09D00B4BB0
:100C10001B68FB60094B00221A60FB6878689847E4
:100C200002E07B6800221A701037BD4680BD00BF0D
:100C300050010020600B00205409002054010020C6
:100C400080B582B000AF7860314B1B78082B01D99A
:100C5000012358E07B682F4A934209D07B682E4AD3
:100C6000934205D0642000F043FEFFF7F1FDFEE75C
:100C70007B681B78012B08D17B689B88002B04D0F4
:100C80007B689B88B3F5817F05D3642000F030FE3C
:100C9000FFF7DEFDFEE7214B1B68002B05D064202B
:100CA00000F026FEFFF7D4FDFEE7194B1B78002B62
:100CB00007D0002B20DB042B1EDC184A7B68136056
:100CC00020E0134B01221A70154A7B681360144B05
:100CD0001B689A79134B1A70114B1B68DA79124B07
:100CE0001A70124B1B78002B05D0104B00221A7083
:100CF00000F0BEF906E005E0642000F0F9FDFFF722
:100D0000A7FDFEE7002318460837BD4680BD00BF9B
:100D100050010020600B0020540900204C010020ED
:100D20005C0B0020680D0020500900205C010020B1
:100D300080B485B000AF7860064B01221A70A02302
:100D4000FB60FB6883F311881437BD465DF8047BB4
:100D5000704700BF5D01002080B582B000AF094B35
:100D60001B78002B00D109E0064B00221A7000F01E
:100D70000BF800237B607B6883F311880837BD463E
:100D800080BD00BF5D01002080B582B000AF6A4B1E
:100D900010229A61694B1B78082B00D9C8E0674B79
:100DA0001B78022B0DD1654B03221A70644B1B7804
:100DB000002B05D0624B00221A7000F07FF9B7E0DB
:100DC000B6E05E4B1B78042B3FD15E4B1B68002BBB
:100DD00009D05D4B1B68002B05D1642000F088FD15
:100DE000FFF736FDFEE7594B1B687B60564B1B68CF
:100DF000002B1DD0514B01221A70534B1B68534AD4
:100E00001360514B00221A60504B1B689A79504B6B
:100E10001A704E4B1B68DA794E4B1A70484B1B7890
:100E2000002B0ED0464B00221A7000F021F908E08A
:100E3000424B00221A70484B1B68002B01D000F077
:100E4000AFF87868FFF7C8FE72E03C4B1B78062BC2
:100E50001ED13E4B1B689B88002B05D03B4B1B686B
:100E60009B88B3F5817F05D3642000F041FDFFF737
:100E7000EFFCFEE7314B07221A70314B1B78002B39
:100E800005D02F4B00221A7000F088F950E04FE097
:100E90002A4B1B78082B45D1284B00221A702E4B69
:100EA0001B68002B05D1642000F022FDFFF7D0FC69
:100EB000FEE7264B1B689B79022B0FD1234B1B6847
:100EC000DB79012B0AD1214B1B681846FFF784FE02
:100ED000214B00221A60FFF7AFFD29E01B4B1B6876
:100EE0009B791A461A4B1B78534003F07F03002B63
:100EF00006D1164B1B68DA79164B1B789A4205D03F
:100F0000642000F0F5FCFFF7A3FCFEE7124B1B6822
:100F10003B60114B00221A600C4B1A683B6810466C
:100F2000984705E0642000F0E3FCFFF791FCFEE742
:100F30000837BD4680BD00BF0000024050010020C0
:100F40005C010020540100204C0100205C0B0020BB
:100F5000680D0020500900205801002080B582B0A3
:100F600000AF78600C4B1B78082B01D901230FE0F0
:100F70000A4B1B68002B05D0642000F0B9FCFFF77A
:100F800067FCFEE7054A7B68136000F009F803463A
:100F900018460837BD4680BD50010020580100208A
:100FA00080B500AF114B1B78082B01D901231BE042
:100FB0000E4B1B78042B05D9642000F099FCFFF739
:100FC00047FCFEE7094B1B78002B0CD1074B052291
:100FD0001A70074B1B78002B05D0054B00221A70A6
:100FE0000448FFF795FD0023184680BD50010020FE
:100FF0005C0100201511000880B500AF194B1B786B
:10100000082B00D92DE0174B1B78072B23D801A202
:1010100052F823F0351000083D1000085710000862
:101020004310000857100008491000085710000826
:10103000511000080C4B01221A7012E000F018F851
:101040000FE000F03BF80CE00848FFF761FD08E016
:1010500000F0A4F805E0642000F04AFCFFF7F8FB7C
:10106000FEE780BD500100205C0100201511000842
:1010700080B500AF0C4B02221A700C4B4FF480125B
:101080009A610B4B1B6804330A4819460A4A02232B
:1010900004F080FA0346002B05D0642000F028FC01
:1010A000FFF7D6FBFEE780BD5001002000000240A4
:1010B0005C0B00206C0D00204C09002080B500AFB7
:1010C000104B04221A70104B4FF480129A610F4B90
:1010D0001B68991D0D4B1B689A1D0C4B1B689B8848
:1010E000022B38BF02239BB2094804F053FA03468F
:1010F000002B05D0642000F0FBFBFFF7A9FBFEE707
:1011000080BD00BF50010020000002405C0B0020A9
:101110006C0D002080B582B000AF78601A4B1B7850
:10112000082B00D92CE0184B1B78052B05D0642028
:1011300000F0DEFBFFF78CFBFEE7134B06221A7074
:10114000124A7B681360114B1B6800229A80104B77
:101150004FF480129A610F4B00221A600B4B1B68F0
:1011600004330D480B491A46022304F013FA0346D0
:10117000002B05D0642000F0BBFBFFF769FBFEE706
:101180000837BD4680BD00BF500100205C0B002029
:10119000000002404C0900206C0D002080B500AF1B
:1011A000104B08221A70104B4FF480129A610F4BAB
:1011B0001B68991D0D4B1B689A1D0C4B1B689B8867
:1011C000022B38BF02239BB2094804F0E3F903461F
:1011D000002B05D0642000F08BFBFFF739FBFEE706
:1011E00080BD00BF50010020000002405C0B0020C9
:1011F0006C0D002080B582B000AF7860064B1B7884
:10120000082B00D905E0642000F072FBFFF720FBFB
:10121000FEE70837BD4680BD5001002080B582B092
:1012200000AF7860FFF72CFB0346002B01D00123B1
:1012300006E0054A7B6813600448FFF769FC034633
:1012400018460837BD4680BDE40D00205112000845
:1012500080B582B000AF78607B6801229A807B689D
:1012600001229A717B680022DA717868FFF7E8FC46
:101270000346002B0ED17868FFF7AEFC0A48FFF753
:101280006DFE0346002B04D0084B1B6801209847D5
:1012900007E006E07868FFF79FFC044B1B6801201D
:1012A00098470837BD4680BDB1120008E40D002004
:1012B00080B582B000AF7860FFF7E2FA0346002BFA
:1012C00000D01EE07B68002B04D10F4B1B6801206F
:1012D000984716E07B689B88022B03D17B681B7ABA
:1012E000002B07D07868FFF777FC074B1B680120BD
:1012F000984706E07868FFF76FFC034B1B680020F7
:1013000098470837BD4680BDE40D002080B584B005
:1013100000AF7860FFF7B4FA0346002B01D0012339
:101320001FE0124A7B681360FFF72EFCF860FB6831
:10133000002B01D1012314E0FB6801229A80FB6895
:1013400001229A71FB680122DA71F868FFF778FCD4
:101350000346002B04D10648FFF700FE034600E0D9
:10136000012318461037BD4680BD00BFDC0D0020AC
:101370007513000880B584B000AF7860FFF780FA7D
:101380000346002B00D022E07B68002B06D1114BD6
:101390001B68002000210022984718E07B689B888A
:1013A000052B06D00B4B1B6800200021002298471C
:1013B0000DE07B6808331B68FB607B680C331B689F
:1013C000BB60044B1B687868F968BA6898471037A7
:1013D000BD4680BDDC0D002080B586B000AFF86052
:1013E000C7E90023FFF74CFA0346002B01D0012385
:1013F00033E01C4B00221A601B4B00221A701B4A60
:101400007B6A13601A4AFB681360FFF7BDFB7861C3
:101410007B69002B01D101231FE07B6907229A80A1
:101420007B6901229A717B690222DA717B6903F17F
:101430000801D7E90023C1E900237B6910333A6A28
:101440001A607869FFF7FCFB0346002B04D10948BA
:10145000FFF784FD034600E0012318461837BD4618
:1014600080BD00BFC80D0020D80D0020EC0D00206D
:10147000E40D0020B112000880B582B000AF7860A2
:10148000FFF7FEF90346002B01D0012321E0134AA8
:101490007B681360124B1B78002B01D0002318E0EF
:1014A0000F4B01221A700F4B1B68002B0DD00B4BFA
:1014B0001B68002B09D00B4B1B68184600F016F870
:1014C000084B00221A60002303E00748FFF746FD9F
:1014D000034618460837BD4680BD00BFE80D002012
:1014E000D80D0020C80D0020ED14000880B584B090
:1014F00000AF7860254B00221A70FFF7C1F9034650
:10150000002B00D03EE0224B1B68002B03D1214A68
:101510007B68136036E07B68002B05D11C4B1B6891
:101520000020002198472DE07B689B88013B9BB2FF
:101530005B00FB817B689B79DBB25BB2002B08DA36
:101540007B689B88012B04D9FA89134B1B689A424C
:1015500005D90F4B1B6800200021984712E00E4B65
:101560001A68FB89D31A0C4A1360094B1B68FA8965
:10157000786811469847084B1B68002B02D0002062
:10158000FFF77AFF1037BD4680BD00BFD80D0020A1
:10159000E80D0020C80D0020EC0D002080B584B0BF
:1015A00000AFF860C7E90023FFF76AF90346002B94
:1015B00001D001230EE00949D7E90023C1E9002346
:1015C000074ABB691360074AFB6813600648FFF7C8
:1015D0009FFA034618461037BD4680BDD00D002047
:1015E000E00D0020E40D0020ED15000880B582B06C
:1015F00000AF78607B6807229A807B6801229A712D
:101600007B680322DA717B6803F10801144BD3E98C
:101610000023C1E900237B681033124A12681A6064
:101620007868FFF70DFB0346002B0ED17868FFF7B3
:10163000D3FA0D48FFF792FC0346002B04D00B4B66
:101640001B680120984707E006E07868FFF7C4FAB6
:10165000064B1B68012098470837BD4680BD00BF78
:10166000D00D0020E00D002071160008E40D0020D0
:1016700080B584B000AF7860FFF702F90346002B15
:1016800000D026E07B68002B04D1134B1B6801209F
:1016900098471EE07B689B88022B07D17B681B7AEA
:1016A000002B0BD07B681B7A022B07D07868FFF7E2
:1016B00093FA094B1B68012098470AE07B681B7A64
:1016C000FB737868FFF788FA034B1B68FA7B1046B8
:1016D00098471037BD4680BDE40D002080B582B02C
:1016E00000AF78603960FFF7CBF80346002B01D0DC
:1016F000012317E03B6803F00103002B01D0012315
:1017000010E03B685B089BB201339AB27B689A8019
:101710007B6881229A717B680322DA717868FFF70F
:101720008FFA034618460837BD4680BD80B500AF26
:1017300000F00EF806F0CCF900F056F800F0C6F80C
:10174000FFF73CF8FFF746F8FFF706FBFCE700BFA2
:1017500080B592B000AF224A214B1B6C43F08053FE
:101760001364204A1F4B1B6823F4404343F4004397
:1017700013600123BB610123FB6102233B634FF430
:1017800080037B630823BB634FF4A873FB630423CC
:101790003B6407237B6407F11803184604F082FAC0
:1017A0000346002B00D0FEE70D237B600223BB60C5
:1017B0000023FB604FF4A0533B614FF480537B61E7
:1017C0003B1D1846022104F051FC0346002B00D0BB
:1017D000FEE7042006F060F94837BD4680BD00BF33
:1017E000003802400070004080B586B000AF324A39
:1017F000314B1B6B43F0010313632F4A2E4B1B6BC2
:1018000043F0020313632C4A2B4B1B6B43F004037E
:101810001363294A284B1B6B43F00803136341F6FB
:10182000FF737B600023BB600123FB6000233B61EF
:1018300000237B613B1D2148194605F091FE4FF6C0
:10184000E7737B603B1D1E48194605F089FE4FF685
:10185000FF737B603B1D1B48194605F081FE3B1D55
:101860001948194605F07CFE10237B600323BB60FA
:101870003B1D1448194605F073FE4FF480537B60FE
:101880000123BB600023FB603B1D0E48194605F099
:1018900067FE0C4B4FF480529A6120237B603B1D06
:1018A0000748194605F05CFE054B4FF400129A619B
:1018B0001837BD4680BD00BF00380240000002401E
:1018C0000004024000080240000C024080B500AF56
:1018D000064B4FF080529A614FF4FA7006F04AF9C5
:1018E000024B4FF480529A6180BD00BF0008024055
:1018F00080B483B000AF0346FB80094AFB881380A5
:10190000FB88002B06D1074B00221A70064B4FF4C0
:1019100080529A610C37BD465DF8047B704700BF6A
:101920005E010020620100200008024080B400AF88
:10193000144B1B88002B21D0134B1B8801339AB208
:10194000114B1A80104B1A880E4B1B889A4215D3E4
:101950000D4B00221A800D4B1B78002B07D00B4B30
:1019600000221A700A4B4FF480529A6106E0074B2E
:1019700001221A70064B4FF080529A61BD465DF805
:10198000047B70475E01002060010020620100209E
:101990000008024080B500AF06F0D2F8FFF7C6FF9E
:1019A00080BD00BF80B500AF014804F021FF80BDBD
:1019B0007403002080B500AF024B08225A61FFF784
:1019C0001BFB80BD003C014080B500AF054B2022D1
:1019D0009A61054803F074FE024B4FF400129A61BD
:1019E00080BD00BF000402406C0D002080B500AF38
:1019F0004FF0FF300221002206F018F880BD00BF32
:101A000080B588B000AF78607B681B68234A93423A
:101A100040D1234A224B5B6C43F480535364E02350
:101A2000FB6002233B6102237B610123BB61052331
:101A3000FB6107F10C031B48194605F091FD194B9A
:101A400010229A611023FB6001233B6100237B611C
:101A500007F10C031348194605F082FD0823FB60CB
:101A6000114B3B6101237B6107F10C030D481946C3
:101A700005F076FD09200A21002205F0D7FF092094
:101A800005F0F0FF23200821002205F0CFFF2320DE
:101A900005F0E8FF2037BD4680BD00BF00300140A3
:101AA00000380240000002400000211080B584B0E0
:101AB00000AFF860B9601346FB80FB680222C3F8F0
:101AC000F421FA88FB689A61FA88FB68DA61FB887E
:101AD000F8680021BA68FEF729FE0023184610377F
:101AE000BD4680BD80B584B000AFF860B9601346D4
:101AF000FB80FB88F8680021BA68FEF717FE002318
:101B000018461037BD4680BD80B584B000AFF86080
:101B1000B9601346FB80FB88F8680021BA68FEF7BD
:101B20001FFE002318461037BD4680BD80B582B029
:101B300000AF78607B680422C3F8F4217868002144
:101B400000220023FEF7F2FD002318460837BD46A9
:101B500080BD00BF80B582B000AF78607B68052291
:101B6000C3F8F4217868002100220023FEF7F8FD75
:101B7000002318460837BD4680BD00BF80B584B03D
:101B800000AF786039600023FB733B685B78092BFA
:101B900039D801A252F823F0E91B0008FD1B000808
:101BA000071C0008F31B0008071C0008CB1B0008DB
:101BB000C11B0008071C0008DF1B0008D51B00081C
:101BC0007868396800F036F922E07868396800F002
:101BD0002DFA1DE07868396800F066FA18E0786838
:101BE000396800F0EBFA13E07868396800F018FB08
:101BF0000EE07868396800F03DFB09E078683968E4
:101C000000F052FB04E07868396800F0B1FB00BFD7
:101C1000FB7B18461037BD4680BD00BF80B584B041
:101C200000AF786039600023FB737B6893F8FC3168
:101C3000032B1CD13B689B88DBB2012B11D87B683E
:101C4000D3F814329B687868396898473B68DB881A
:101C5000002B0BD1FB7B002B08D17868FFF766FFC8
:101C60000AE07868396800F083FB05E004E07868F2
:101C7000396800F07DFB00BF002318461037BD46D1
:101C800080BD00BF80B584B000AF786039600023AC
:101C9000FB733B689B88BB733B681B7803F0600356
:101CA000202B08D17B68D3F814329B687868396898
:101CB00098470023B9E03B685B78012B39D0032BB0
:101CC00002D0002B6AD0AFE07B6893F8FC31022B86
:101CD00002D0032B0DD026E0BB7B002B08D0BB7BB2
:101CE000802B05D0BB7B78681946FEF7B7FC1FE058
:101CF0001EE03B685B88002B0AD1BB7B002B07D022
:101D0000BB7B802B04D0BB7B78681946FEF7A6FC12
:101D10007B68D3F814329B6878683968984778688C
:101D2000FFF704FF04E07868396800F021FB00BF8A
:101D30007AE07B6893F8FC31022B02D0032B0DD0A4
:101D400026E0BB7B002B08D0BB7B802B05D0BB7B68
:101D500078681946FEF782FC1FE01EE03B685B884E
:101D6000002B14D1BB7B03F07F03002B0BD0BB7B7C
:101D700078681946FEF786FC7B68D3F814329B68B6
:101D80007868396898477868FFF7D0FE05E004E086
:101D90007868396800F0ECFA00BF45E07B6893F89A
:101DA000FC31022B02D0032B0CD037E0BB7B03F0BD
:101DB0007F03002B05D0BB7B78681946FEF74EFCED
:101DC00031E030E0BB7B5BB2002B08DABB7B03F079
:101DD0007F0301331B017A681344043307E0BB7BA4
:101DE00003F07F0310331B017A6813440433BB6094
:101DF000BB7B78681946FEF759FC0346002B03D0DD
:101E0000BB6801221A6002E0BB6800221A60BB684E
:101E1000786819460222FFF749FE04E078683968BD
:101E200000F0A6FA00BF00BFFB7B18461037BD4686
:101E300080BD00BF80B584B000AF786039603B687A
:101E40005B881B0A9BB2013B062B00F2D18001A2EA
:101E500052F823F0711E00088B1E0008CB1E0008EC
:101E6000F11F0008F11F00089D1F0008C31F000894
:101E70007B68D3F810321B687A68117C07F10A027C
:101E8000084611469847F860B7E07B681B7C002B3A
:101E90000DD17B68D3F81432DB6A07F10A021046D1
:101EA0009847F860FB68013302221A70A5E07B684E
:101EB000D3F814321B6B07F10A0210469847F860FA
:101EC000FB68013302221A7097E03B685B88DBB243
:101ED000052B5DD801A252F823F000BFF51E0008C3
:101EE0000F1F0008291F0008431F00085D1F00087E
:101EF000771F00087B68D3F810325B687A68117C22
:101F000007F10A02084611469847F86045E07B68E9
:101F1000D3F810329B687A68117C07F10A020846F0
:101F200011469847F86038E07B68D3F81032DB68D8
:101F30007A68117C07F10A02084611469847F86052
:101F40002BE07B68D3F810321B697A68117C07F1AB
:101F50000A02084611469847F8601EE07B68D3F8ED
:101F600010325B697A68117C07F10A020846114653
:101F70009847F86011E07B68D3F810329B697A6863
:101F8000117C07F10A02084611469847F86004E000
:101F90007868396800F0ECF944E02EE07B681B7C3F
:101FA000002B09D17B68D3F814329B6B07F10A022E
:101FB00010469847F86020E07868396800F0D8F952
:101FC00030E07B681B7C002B0DD17B68D3F814328A
:101FD0005B6B07F10A0210469847F860FB68013313
:101FE00007221A7009E07868396800F0C1F919E031
:101FF0007868396800F0BCF914E07B89002B11D0B7
:102000003B68DB88002B0DD03B68DA887B899342E4
:1020100028BF13469BB27B817B897868F9681A4692
:10202000FFF744FD1037BD4680BD00BF80B584B0CA
:1020300000AF786039603B689B88002B2DD13B68EE
:10204000DB88002B29D13B685B88DBB203F07F0380
:10205000FB737B6893F8FC31032B04D178683968F3
:1020600000F086F918E07B68FA7B83F8FE21FB7BA1
:1020700078681946FEF746FB7868FFF757FDFB7B4B
:10208000002B04D07B68022283F8FC2104E07B68EB
:10209000012283F8FC2104E003E07868396800F04D
:1020A00067F91037BD4680BD80B582B000AF78605B
:1020B00039603B685B88DAB23F4B1A703E4B1B7845
:1020C000012B04D97868396800F052F970E07B6818
:1020D00093F8FC31022B02D0032B23D063E0364B64
:1020E0001B78002B1AD0344B1B781A467B685A6039
:1020F0007B68032283F8FC212F4B1B7878681946F4
:1021000000F012FA0346022B04D17868396800F017
:102110002FF94DE07868FFF709FD49E07868FFF78F
:1021200005FD45E0244B1B78002B12D17B68022271
:1021300083F8FC21204B1B781A467B685A601E4BA3
:102140001B787868194600F00FFA7868FFF7EEFC04
:1021500028E0194B1B781A467B685B689A421DD0B1
:102160007B685B68DBB27868194600F0FDF9124BBA
:102170001B781A467B685A600F4B1B7878681946A3
:1021800000F0D2F90346022B04D17868396800F0D8
:10219000EFF80DE07868FFF7C9FC03E07868FFF717
:1021A000C5FC05E004E07868396800F0E1F800BF9C
:1021B0000837BD4680BD00BF6301002080B582B0F6
:1021C00000AF786039603B68DB88012B04D0786809
:1021D000396800F0CDF81FE07B6893F8FC31022BE2
:1021E00002D0032B0BD012E07B6800229A607B6840
:1021F0000833786819460122FFF758FC0CE07B6829
:102200000433786819460122FFF750FC04E078682F
:10221000396800F0ADF800BF0837BD4680BD00BF8B
:1022200080B582B000AF786039607B6893F8FC318C
:10223000023B012B15D87B680122DA607B68D3F85A
:102240000432002B05D07B68DB6843F002027B6818
:10225000DA607B680C33786819460222FFF726FCA7
:1022600004E07868396800F083F800BF0837BD469D
:1022700080BD00BF80B582B000AF786039603B6838
:102280005B88012B0DD17B680122C3F804227B6897
:10229000D3F814329B687868396898477868FFF7F4
:1022A00045FC0837BD4680BD80B582B000AF786080
:1022B00039607B6893F8FC31023B012B13D83B68F3
:1022C0005B88012B0ED17B680022C3F804227B6857
:1022D000D3F814329B687868396898477868FFF7B4
:1022E00025FC05E004E07868396800F041F800BF9B
:1022F0000837BD4680BD00BF80B483B000AF7860B2
:1023000039603B681A787B681A703B685A787B683A
:102310005A703B6802331B789AB23B6803331B78D0
:102320009BB21B029BB213449AB27B685A803B68F3
:1023300004331B789AB23B6805331B789BB21B02AF
:102340009BB213449AB27B689A803B6806331B7831
:102350009AB23B6807331B789BB21B029BB21344B3
:102360009AB27B68DA800C37BD465DF8047B704713
:1023700080B582B000AF7860396078688021FEF760
:102380006DF978680021FEF769F90837BD4680BD10
:1023900080B586B000AFF860B9607A600023FB7545
:1023A000FB68002B33D0F86800F034F803460133A3
:1023B0009BB25B009AB27B681A80FB7D5A1CFA754F
:1023C0001A46BB6813447A681288D2B21A70FB7D31
:1023D0005A1CFA751A46BB68134403221A7012E09D
:1023E000FB7D5A1CFA751A46BB681A44FB68591CD7
:1023F000F9601B781370FB7D5A1CFA751A46BB688E
:10240000134400221A70FB681B78002BE8D11837A0
:10241000BD4680BD80B485B000AF78600023FB73FB
:1024200005E0FB7B0133FB737B6801337B607B68DA
:102430001B78002BF5D1FB7B18461437BD465DF8A1
:10244000047B704780B584B000AFF860B960134674
:10245000FB71FB68002B01D1022319E0FB6800220D
:10246000C3F81422FB680022C3F81822BB68002BB3
:1024700003D0FB68BA68C3F81022FB68012283F816
:10248000FC21FB68FA791A70F868FEF73BF8002324
:1024900018461037BD4680BD80B485B000AF786067
:1024A00039600023FB733B68002B06D07B683A68D9
:1024B000C3F814220023FB7301E00223FB73FB7BB0
:1024C00018461437BD465DF8047B704780B582B06E
:1024D00000AF78607868FEF75FF800231846083789
:1024E000BD4680BD80B582B000AF78607B68D3F810
:1024F00014325B687A685268D2B27868114698479D
:102500007868FEF759F8002318460837BD4680BDA5
:1025100080B483B000AF7860002318460C37BD4606
:102520005DF8047B704700BF80B584B000AF786071
:102530000B46FB700223FB737B68D3F81432002B2D
:102540000CD07B68D3F814321B68FA78786811468F
:1025500098470346002B01D10023FB73FB7B1846F1
:102560001037BD4680BD00BF80B582B000AF786037
:102570000B46FB707B68D3F814325B68FA78786896
:1025800011469847002318460837BD4680BD00BF56
:1025900080B582B000AF786039607B6803F5027364
:1025A00018463968FFF7A8FE7B680122C3F8F421BA
:1025B0007B68B3F80E321A467B68C3F8F8217B6853
:1025C00093F8083203F01F03012B0BD0022B11D01C
:1025D000002B17D17B6803F5027378681946FFF763
:1025E000CDFA1AE07B6803F5027378681946FFF7A5
:1025F00015FB12E07B6803F5027378681946FFF754
:1026000041FB0AE07B6893F8083223F07F03DBB2DA
:1026100078681946FEF722F800BF002318460837ED
:10262000BD4680BD80B586B000AFF8600B467A60CD
:10263000FB72FB7A002B38D1FB6803F582737B6158
:10264000FB68D3F8F431032B42D17B699A687B692C
:10265000DB689A4214D97B699A687B69DB68D21A75
:102660007B699A607B69DA687B699B68934228BFC3
:1026700013469BB2F86879681A46FFF745FA27E0D7
:10268000FB68D3F814321B69002B0AD0FB6893F85F
:10269000FC31032B05D1FB68D3F814321B69F868B1
:1026A0009847F868FFF742FA12E0FB68D3F8143253
:1026B0009B69002B0CD0FB6893F8FC31032B07D1EE
:1026C000FB68D3F814329B69FA7AF8681146984788
:1026D000002318461837BD4680BD00BF80B586B0C0
:1026E00000AFF8600B467A60FB72FB7A002B6CD16E
:1026F000FB6814337B61FB68D3F8F431022B57D1AC
:102700007B699A687B69DB689A420FD97B699A6812
:102710007B69DB68D21A7B699A607B699B689BB294
:10272000F86879681A46FFF7DDF905E0F8680021D6
:1027300000220023FEF714F87B695B687A69D2688F
:10274000B3FBF2F102FB01F29B1A002B16D17B695D
:102750005A687B69DB689A4210D37B695A68FB68C8
:10276000D3F8F8319A4209D2F86800210022FFF725
:10277000B9F9FB680022C3F8F82105E0F8680021E8
:1027800000220023FDF7ECFFFB68D3F81432DB686E
:10279000002B0AD0FB6893F8FC31032B05D1FB68B2
:1027A000D3F81432DB68F8689847F868FFF7D2F975
:1027B000FB6893F80032012B1AD1F868FFF7A8FEE6
:1027C000FB68002283F8002212E0FB68D3F8143281
:1027D0005B69002B0CD0FB6893F8FC31032B07D10D
:1027E000FB68D3F814325B69FA7AF86811469847A7
:1027F000002318461837BD4680BD00BF80B582B0A3
:1028000000AF78607868002100224023FDF7E4FEE5
:102810007B684022C3F81021786880210022402381
:10282000FDF7DAFE7B6840221A627B68012283F89A
:10283000FC217B68D3F81832002B09D07B68D3F8D1
:1028400014325B687A685268D2B278681146984749
:10285000002318460837BD4680BD00BF80B483B052
:1028600000AF78600B46FB707B68FA781A7400231F
:1028700018460C37BD465DF8047B704780B483B0C2
:1028800000AF78607B6893F8FC217B6883F8FD21BA
:102890007B68042283F8FC21002318460C37BD46D0
:1028A0005DF8047B704700BF80B483B000AF7860F0
:1028B0007B6893F8FD217B6883F8FC210023184690
:1028C0000C37BD465DF8047B704700BF80B582B011
:1028D00000AF78607B6893F8FC31032B0BD17B68E9
:1028E000D3F81432DB69002B05D07B68D3F814329F
:1028F000DB6978689847002318460837BD4680BDD5
:1029000080B483B000AF78600B46FB70002318469C
:102910000C37BD465DF8047B704700BF80B483B0C0
:1029200000AF78600B46FB70002318460C37BD469D
:102930005DF8047B704700BF80B483B000AF78605F
:10294000002318460C37BD465DF8047B704700BF76
:1029500080B582B000AF78607B68012283F8FC21EB
:102960007B68D3F814325B687A685268D2B27868B0
:1029700011469847002318460837BD4680BD00BF62
:1029800080B582B000AF78607B68D3F814329B6A60
:1029900078689847002318460837BD4680BD00BFB9
:1029A00080B584B000AFF8607A603B600B46FB7284
:1029B000814AFB681360814A7B681360804AFB7A16
:1029C0001370804A3B681360FB68D3F818327E4A64
:1029D00013607B681B785A2B00F2DE8001A252F84C
:1029E00023F000BF512B0008992B0008992B0008F9
:1029F000572B0008992B0008992B0008992B0008E9
:102A0000992B0008992B0008992B0008992B000896
:102A1000992B0008992B0008992B0008992B000886
:102A2000992B0008992B0008992B00085D2B0008B2
:102A3000992B0008992B0008992B0008992B000866
:102A4000992B0008992B0008992B00086F2B000880
:102A5000632B0008992B0008992B0008692B0008AC
:102A6000992B0008992B0008992B0008992B000836
:102A70007B2B0008992B0008812B0008992B00085C
:102A8000992B0008872B0008992B00088D2B000834
:102A9000992B0008992B0008992B0008992B000806
:102AA000932B0008992B0008992B0008992B0008FC
:102AB000992B0008992B0008992B0008992B0008E6
:102AC000992B0008992B0008992B0008992B0008D6
:102AD000992B0008992B0008992B0008992B0008C6
:102AE000992B0008992B0008992B0008992B0008B6
:102AF000992B0008992B0008992B0008992B0008A6
:102B0000992B0008992B0008992B0008992B000895
:102B1000992B0008992B0008992B0008992B000885
:102B2000992B0008992B0008992B0008992B000875
:102B3000992B0008992B0008992B0008992B000865
:102B4000992B0008992B0008992B0008752B000879
:102B500000F03CF82CE000F09DFA29E000F09AF833
:102B600026E000F06DFB23E000F06AFB20E000F0BF
:102B70002DFA1DE000F05CFA1AE000F089F917E088
:102B800000F0E0F814E000F06BFB11E000F0B2FCA4
:102B90000EE000F035FE0BE0FB7AF86819460522DE
:102BA000202300F00FFB074B1B684FF0FF309847C6
:102BB0001037BD4680BD00BF000E0020F40D002080
:102BC000F80D0020FC0D0020F00D002080B500AFB6
:102BD000134B1B68DB69002B0FD0124B1A68124B8A
:102BE0001B78104619460522202300F0EBFA0F4B04
:102BF0001B684FF0FF30984710E00B4B1B78002B01
:102C000003D0012000F016F808E00948FEF706FBA3
:102C10000346002B02D0012000F00CF880BD00BF5D
:102C2000F00D0020000E0020F80D0020FC0D00200B
:102C3000352C000880B582B000AF0346FB71FB79EC
:102C4000002B13D00F4B1A680F4B1B7810461946F8
:102C500002223A2300F0B6FA0C4B1B6805221A72C6
:102C60000B4B1B684FF0FF30984707E0074B1B6882
:102C700000225A81064B1B68002098470837BD4642
:102C800080BD00BF000E0020F80D0020F00D0020D8
:102C9000FC0D002080B584B000AFFDF775FF7860B3
:102CA000234B1B687A681A61214B1B687A680832CB
:102CB000DA60204B1B6801331B7803F00103002B03
:102CC00004D01D4BFB6007237B8114E01B4BFB6092
:102CD000FB6804331B789BB205337B81154B1B6863
:102CE00004331B789BB27A899A4204D3114B1B6838
:102CF00004331B787B810E4B1B687A895A810CE068
:102D00007B89013B7B810A4B1B68DA687B89134412
:102D10007A89F9680A4412781A707B89002BEFD1FE
:102D2000074B1B68002098471037BD4680BD00BF89
:102D3000F00D0020F40D0020547E0008DC7D00081A
:102D4000FC0D002080B500AF0548FEF7DFFA034612
:102D5000002B04D000200021002200F003F880BDE9
:102D6000652D000880B584B000AFF860B9607A6066
:102D7000FB68002B0FD1424B1A68424B1B78104660
:102D8000194602223A2300F01DFA3F4B1B684FF010
:102D9000FF30984771E03D4B1B68FA681A613B4B66
:102DA0001B68FA680832DA60384B1B68BA689A66A2
:102DB000364B1B687A6892B2A3F86620334B1B68C7
:102DC000DB68324A1268926E013A120ED2B21A7061
:102DD0002E4B1B68DB6801332C4A1268926E013A55
:102DE000120CD2B21A70294B1B68DB680233274AD7
:102DF0001268926E013A120AD2B21A70234B1B6803
:102E0000DB680333214A1268926ED2B2013AD2B221
:102E10001A701E4B1B68DB6804331C4A1268B2F838
:102E200066201216D2B21A70184B1B68DB68053385
:102E3000164A1268B2F866201214D2B21A70134BF6
:102E40001B68DB680633114A1268B2F86620120A62
:102E500092B2D2B21A700D4B1B68DB6807330B4A73
:102E60001268B2F86620D2B21A70084B1B680822AA
:102E70005A81054B1B68002098471037BD4680BD1E
:102E8000000E0020F80D0020FC0D0020F00D0020A9
:102E900080B500AF0548FEF739FA0346002B04D091
:102EA00000200021002200F003F880BDB12E0008B0
:102EB00080B584B000AFF860B9607A60FB68002B21
:102EC0000FD13E4B1A683E4B1B7810461946022222
:102ED0003A2300F077F93B4B1B684FF0FF309847DF
:102EE00068E0394B1B68FA681A61374B1B68FA684F
:102EF0000832DA60344B1B68DB6800221A70324BF0
:102F00001B68DB68013300221A702F4B1B68DB68DB
:102F1000023300221A702C4B1B68DB680333082233
:102F20001A70294B1B68DB680433BA68013A120E29
:102F3000D2B21A70244B1B68DB680533BA68013AB9
:102F4000120CD2B21A70204B1B68DB680633BA68C9
:102F5000013A120AD2B21A701B4B1B68DB680733A6
:102F6000BA68D2B2013AD2B21A70174B1B68DB684A
:102F7000083302221A70144B1B68DB6809337A6825
:102F8000120CD2B21A70104B1B68DB680A337A68D5
:102F9000120AD2B21A700C4B1B68DB680B337A68CA
:102FA000D2B21A70084B1B680C225A81054B1B6861
:102FB000002098471037BD4680BD00BF000E00209E
:102FC000F80D0020FC0D0020F00D002080B582B02F
:102FD00000AF0823FB80FDF7D7FD3860114B1B685D
:102FE0003A681A610F4B1B683A680832DA600D4B79
:102FF0001B68FA885A810BE0FB88013BFB80094B78
:103000001B68DA68FB881344FA8807498A5C1A70DF
:10301000FB88002BF0D1054B1B6800209847083730
:10302000BD4680BDF00D00205C7E0008FC0D002038
:1030300080B582B000AF0823FB80FDF7A5FD3860A6
:10304000114B1B683A681A610F4B1B683A680832CB
:10305000DA600D4B1B68FA885A810BE0FB88013B54
:10306000FB80094B1B68DA68FB881344FA88074920
:103070008A5C1A70FB88002BF0D1054B1B6800207E
:1030800098470837BD4680BDF00D0020647E0008DB
:10309000FC0D002080B582B000AFFDF775FD3860F3
:1030A000454B1B683A681A61434B1B683A68083203
:1030B000DA600023FB7109E03F4B1B68DA68FB799B
:1030C000134400221A70FB790133FB71FB79112B39
:1030D000F2D9394B1B68DB6870221A70364B1B68BB
:1030E000DB6807330C221A70334B1B6893F864209B
:1030F000314B1B6893F865309A4244D02E4B1B68C5
:10310000DB689A1C2C4B19682B4B1B6893F86430B6
:103110000833DB000B441B79DBB21370264B1B68B2
:10312000DB6803F10C02244B1968234B1B6893F8EE
:1031300064300833DB000B445B7ADBB213701E4B48
:103140001B68DB6803F10D021B4B19681A4B1B68E7
:1031500093F864300833DB000B441B7ADBB2137046
:10316000154B1B6893F864200132D2B283F86420B7
:10317000114B1B6893F86430042B04D10E4B1B6871
:10318000002283F864200C4B1B6812225A810B4BDF
:103190001B6804331B78122B07D8074B1B68074AA0
:1031A00012680432127892B25A81054B1B680020D3
:1031B00098470837BD4680BDF00D0020F40D002073
:1031C000FC0D002080B485B000AF78600846114641
:1031D0001A460346FB700B46BB7013467B707B6838
:1031E000D3F81832FB60FB6893F86530B978FA6859
:1031F0000833DB0013440A461A71FB6893F8653004
:1032000018467B781B021946FA6800F10803DB00B8
:1032100013449960FB6893F865300133DAB2FB68B8
:1032200083F86520FB6893F86530042B03D1FB68B5
:10323000002283F865201437BD465DF8047B704793
:1032400080B500AF044B1B6800225A81034B1B68FA
:103250000020984780BD00BFF00D0020FC0D00202D
:1032600080B582B002AF5A4B1B681B7A002B40F02E
:10327000A280574B1B6893F82030DBB25BB2002B67
:1032800011DB544B1A68524B1B6893F821301046DF
:10329000194605222023FFF795FF4F4B1B684FF07F
:1032A000FF30984791E04A4B1B684C4A1268023243
:1032B00012781106494A1268033212781204114337
:1032C000464A12680432127812020A4343490968D6
:1032D000053109780A43DA663D4B1B683F4A12689C
:1032E00007321278120291B23C4A12680832127800
:1032F00092B20A4392B292B2A3F87020344B1B6888
:10330000DA6E334B1B68B3F870301046194600F084
:10331000B9FA0346002B11DA2E4B1A682C4B1B68A6
:1033200093F821301046194605222023FFF74AFF63
:10333000294B1B684FF0FF30984746E0244B1B6831
:10334000DB69234A1268B2F870201146204A1268DD
:10335000B2F8662002FB01F2934211D01D4B1A68AD
:103360001B4B1B6893F82130104619460522202379
:10337000FFF728FF184B1B684FF0FF30984724E0F9
:10338000134B1B68DB6E1A464FF0000310490968A7
:10339000B1F8701008460E490968C969009001919A
:1033A0000F48FEF719F80346002B03D0012000F068
:1033B0001BF80AE009E00B48FEF75EF80346002B15
:1033C00003D00020002100F043F8BD4680BD00BFBF
:1033D000F00D0020000E0020FC0D0020F40D002058
:1033E000E93300085134000880B582B000AF0346CD
:1033F000FB71FB79002B0FD0104B1A68104B1B7818
:103400001046194602223A23FFF7DCFE0D4B1B68DB
:103410004FF0FF3098470DE00B4B1B6802221A72E9
:103420000A48FEF729F80346002B03D000200021AC
:1034300000F00EF80837BD4680BD00BF000E00202A
:10344000F80D0020FC0D0020F00D00205134000884
:1034500080B582B000AF78600B467B807B68002B24
:103460000FD1204B1A68204B1B78104619460422B6
:103470001123FFF7A7FE1D4B1B684FF0FF30984745
:103480002DE01B4B1B681B69002B00D0FEE7184B7F
:103490001B687A681A61164B1B687A680832DA6012
:1034A000104B1968124B1B68DA687B88084681212B
:1034B000FDF73CF90E4B1B680D4A1268D16B7A88F8
:1034C0008A1ADA630A4B1B68DB6B002B03D1084BAB
:1034D0001B6803221A72054B1B68002098470837A7
:1034E000BD4680BD000E0020F80D0020FC0D002020
:1034F000F00D002080B584B002AF7B4B1B681B7AB7
:10350000002B40F09D80784B1B6893F82030DBB295
:103510005BB2002B11DA754B1A68734B1B6893F87A
:1035200021301046194605222023FFF74BFE704B31
:103530001B684FF0FF309847D2E06B4B1B686D4A19
:1035400012680232127811066A4A1268033212783F
:1035500012041143674A12680432127812020A43B5
:1035600064490968053109780A43DA665E4B1B68CD
:10357000604A126807321278120291B25D4A1268EC
:103580000832127892B20A4392B292B2A3F8702033
:10359000554B1B68DA6E544B1B68B3F870301046FD
:1035A000194600F06FF90346002B11DA4F4B1A68E9
:1035B0004D4B1B6893F821301046194605222023F5
:1035C000FFF700FE4A4B1B684FF0FF30984787E03B
:1035D000454B1B68DB69444A1268B2F870201146FB
:1035E000414A1268B2F8662002FB01F2934211D000
:1035F0003E4B1A683C4B1B6893F821301046194625
:1036000005222023FFF7DEFD394B1B684FF0FF300A
:10361000984765E0344B1B68DB6E1A464FF0000399
:1036200031490968B1F8701000913348FDF7B6FFD1
:103630000346002B03D0012000F064F850E04FE077
:10364000294B1B68DB6BB3F5007F28BF4FF4007379
:103650007B60254B1B681B6918467968FEF73EF8AE
:103660000346002B0FD0214B1A68244B1B781046C1
:10367000194604220323FFF7A5FD1D4B1B684FF0DD
:10368000FF3098472CE0184B1B68174A1268D16B23
:103690007A688A1ADA63144B1B68DB6B002B0AD139
:1036A000124B1B681846002100F0C0FA104B1B6833
:1036B0000020984714E01248FDF72AFA0346002B31
:1036C0000ED00A4B1A680D4B1B7810461946022281
:1036D0003A23FFF777FD064B1B684FF0FF30984702
:1036E0000837BD4680BD00BFF00D0020000E002051
:1036F000FC0D0020F40D002005370008F80D002017
:10370000A937000880B582B000AF0346FB71FB7992
:10371000022B0FD11F4B1A681F4B1B7810461946FE
:1037200002222723FFF74EFD1C4B1B684FF0FF3092
:1037300098472BE0FB79002B0FD0164B1A68164BDD
:103740001B781046194602223A23FFF73BFD134B24
:103750001B684FF0FF30984718E0114B1B6801229F
:103760001A721048FDF7D4F90346002B0ED0094B0E
:103770001A68094B1B781046194602223A23FFF7B4
:1037800021FD064B1B684FF0FF3098470837BD46B8
:1037900080BD00BF000E0020F80D0020FC0D0020B1
:1037A000F00D0020A937000880B582B000AF786026
:1037B000104B1B687A681A610E4B1B687A680832D6
:1037C000DA600D4B19680B4B1B68DA68094B1B68F4
:1037D000DB6BB3F5007F28BF4FF400739BB2084644
:1037E0000121FCF7BDFF054B1B68002098470837F7
:1037F000BD4680BDF00D0020000E0020FC0D002015
:1038000080B500AF1A4B1B6801331B7803F002032D
:10381000002B0FD0174B1A68174B1B781046194610
:1038200005222423FFF7CEFC144B1B684FF0FF301A
:1038300098471BE0124B1B68DA6E114B1B68B3F8FC
:1038400070301046194600F01DF80346002B05DACB
:103850000A4B1B684FF0FF30984707E0084B1B6886
:1038600000225A81054B1B680020984780BD00BF8D
:10387000F40D0020000E0020F80D0020FC0D0020AB
:10388000F00D002080B582B000AF78600B467B80E1
:103890000F4B1B689A6E7B689A4207D37A887B68C5
:1038A0001A440B4B1B689B6E9A420BD9094B1A6842
:1038B000094B1B781046194605222123FFF782FC8D
:1038C000FF2300E000235BB218460837BD4680BDE9
:1038D000F00D0020000E0020F80D002080B584B00F
:1038E00000AF78607B68D3F81832FB60FB68002279
:1038F0001A72FB6800225A72FB68002283F8652066
:10390000FB68002283F8642078680121FCF792FEAE
:1039100078688121FCF78EFEFB68143378680121FA
:103920001A461F23FCF71CFF1037BD4680BD00BFA1
:1039300080B584B000AF78607B68D3F81832FB6044
:10394000FB6800221A72FB6801225A72FB6814336A
:10395000786801211A461F23FCF702FF1037BD4685
:1039600080BD00BF80B485B000AF78607B68D3F8BD
:103970001832FB60FB6800221A721437BD465DF8EE
:10398000047B704780B584B000AF78600B46FB7055
:103990007B68D3F81832FB60FB681B7A022B04D0DB
:1039A000022B16DB042B14DC0EE00C4A7B68136040
:1039B000FB6893F82120FB682333786811461A4688
:1039C000074BFEF7EDFF05E07868002100F02EF9C7
:1039D00000E000BF1037BD4680BD00BF040E0020D0
:1039E000E539000880B582B000AF0346FB7197F956
:1039F0000730002B05DA044B1B681846012100F044
:103A000015F90837BD4680BD040E002080B584B08E
:103A100000AF78600B46FB707B68D3F81832FB6010
:103A2000FB681B7A002B02D0012B04D012E07868CF
:103A300000F02CF80EE0094A7B681360FB6893F8ED
:103A40002120FB682333786811461A46044BFEF7A1
:103A5000A7FF00BF1037BD4680BD00BF040E002089
:103A6000653A000880B582B000AF0346FB7197F954
:103A70000730002B05DA044B1B681846012100F0C3
:103A8000D5F80837BD4680BD040E002080B584B04F
:103A900000AF78607B68D3F81832FB60FB689A69E6
:103AA000FB689A63FB68DA69FB68DA63786801216E
:103AB000FCF770FE03461F2B13D1FB685B691B4AA2
:103AC00093420ED1FB6893F82130012B09D8FB6893
:103AD00093F82230002B04D0FB6893F82230102B8F
:103AE0000FD9FB6893F82130786819460522202306
:103AF000FFF768FBFB6802225A72786800F0C2F890
:103B000010E00B4A7B6813600A4AFB681360FB688D
:103B100093F82120FB682333786811461A46064B38
:103B2000FEF73EFF1037BD4680BD00BF55534243F0
:103B3000040E0020080E00203D3B000880B582B036
:103B400000AF0346FB7197F90730002B11DA214BC8
:103B50001B681B7A052B06D11F4B1B6818460121D9
:103B600000F064F832E01C4B1B68184600F08AF83D
:103B70002CE0184B1B681B7A022B27D0154B1B68B7
:103B80001B7A012B22D0134B1B681B7A032B1DD0F1
:103B9000104B1B685B89002B0DD00F4B19680D4B28
:103BA0001B68DA680B4B1B685B89084611461A468E
:103BB00000F014F80AE0074B1B685B89002B05D165
:103BC000054B1B681846002100F030F80837BD4649
:103BD00080BD00BF080E0020040E002080B586B016
:103BE00000AFF860B9601346FB80FB68D3F8183269
:103BF0007B61FA887B69DB69934228BF1346FB80AF
:103C00007B69DA6BFB88D21A7B69DA637B690022F5
:103C100083F840207B6904221A72FB88F8688121AE
:103C2000BA68FCF783FD1837BD4680BD80B584B007
:103C300000AF78600B46FB707B68D3F81832FB60EE
:103C4000FB680F4A5A63FB68FA7883F84020FB68E8
:103C500000221A72FB6800221A61FB68343378680C
:103C600081211A460D23FCF761FDFB681433786847
:103C700001211A461F23FCF773FD1037BD4680BD96
:103C80005553425380B584B000AF78607B68D3F859
:103C90001832FB60FB6893F82030002B0BD1FB68D7
:103CA000DB69002B07D0FB685B7A002B03D17868B7
:103CB0000121FCF7D3FC78688121FCF7CFFCFB687D
:103CC0005B7A022B07D1FB681433786801211A460E
:103CD0001F23FCF745FD1037BD4680BD80B584B07D
:103CE00000AF78600B46FB707B68D3F81832FB603E
:103CF000FB685B7A022B07D178688121FCF7AEFC68
:103D0000FB6800225A720BE0FB785BB2002B07DAEB
:103D1000FB685B7A012B03D078680121FFF786FFEF
:103D20001037BD4680BD00BF80B584B000AF78605D
:103D30000B46FB700023FB817B681B7C002B0ED1A4
:103D40007868012102224FF40073FCF745FC786883
:103D5000812102224FF40073FCF73EFC0BE07868EF
:103D6000012102224023FCF737FC786881210222DE
:103D70004023FCF731FC742003F068FF03461A4629
:103D80007B68C3F818227B68D3F81832002B02D165
:103D90000123FB8109E07868FFF7A0FD7B68D3F879
:103DA000183200221A610023FB81FB89DBB218461E
:103DB0001037BD4680BD00BF80B582B000AF7860CF
:103DC0000B46FB7078680121FCF720FC78688121A4
:103DD000FCF71CFC7868FFF7C5FD7B68D3F8183248
:103DE000002B09D07B68D3F81832184603F036FF51
:103DF0007B680022C3F81822002318460837BD4606
:103E000080BD00BF80B584B000AF786039607B684A
:103E1000D3F81832FB603B681B7803F06003002B7B
:103E200046D0202B00D09DE03B685B78FE2B02D073
:103E3000FF2B1ED035E03B685B88002B13D13B681D
:103E4000DB88012B0FD13B681B78DBB25BB2002B08
:103E500009DAFB6800221A60FB68786819460122BB
:103E6000FDF724FE23E078683968FEF781FA022323
:103E700079E03B685B88002B0DD13B68DB88002B29
:103E800009D13B681B78DBB25BB2002B03DB78689F
:103E9000FFF74EFD0BE078683968FEF769FA0223F8
:103EA00061E078683968FEF763FA02235BE059E065
:103EB0003B685B780A2B04D00B2B0AD0012B0FD068
:103EC0004FE0FB680433786819460122FDF7EEFDE8
:103ED00047E03B685B88DBB21A46FB685A6040E00B
:103EE0003B689B88DBB278681946FCF7A3FB3B680C
:103EF0009B88DBB278681946FCF788FB3B689B8897
:103F0000DBB25BB2002B12DA7B681B7C002B07D183
:103F10007868812102224FF40073FCF75DFB18E002
:103F20007868812102224023FCF756FB11E07B6870
:103F30001B7C002B07D17868012102224FF400730B
:103F4000FCF74AFB05E07868012102224023FCF7D8
:103F500043FB3B689B88DBB278681946FFF7BEFEDF
:103F600000BF00BF002318461037BD4680BD00BF0C
:103F700080B582B000AF78600B46FB70FB78786844
:103F80001946FFF7FFFC002318460837BD4680BDE1
:103F900080B582B000AF78600B46FB70FB78786824
:103FA0001946FFF733FD002318460837BD4680BD8C
:103FB00080B582B000AF78607B68D3F81832002BF0
:103FC00011D07B68D3F818321B69002B0BD07B68AB
:103FD000D3F818321B691846FCF7FEFD7B68D3F84E
:103FE000183200221A61002318460837BD4680BDEA
:103FF00080B483B000AF78607B6820221A80034BC6
:1040000018460C37BD465DF8047B704770000020F1
:1040100080B483B000AF78607B6820221A80034BA5
:1040200018460C37BD465DF8047B704790000020B1
:1040300080B483B000AF78607B6820221A80034B85
:1040400018460C37BD465DF8047B7047B000002071
:1040500080B483B000AF78607B680A221A80034B7B
:1040600018460C37BD465DF8047B7047D000002031
:1040700084B080B582B000AF786007F1140080E8AA
:104080000E00BB6A012B20D17B689B6B23F480322E
:104090007B689A637B68DB6823F4840323F0400326
:1040A0007A68D3607B68DB6823F440127B68DA604F
:1040B0003B6C012B05D17B68DB6843F480127B6885
:1040C000DA60786801F0CCF90CE07B68DB6843F0DB
:1040D00040027B68DA60786801F0C2F97B684FF4CF
:1040E00080329A633B6A012B0BD17B689B6843F05B
:1040F0000C027B689A607B689B6843F020027B68B7
:104100009A60002318460837BD46BDE8804004B0D9
:10411000704700BF80B483B000AF78607B689B6855
:1041200043F001027B689A60002318460C37BD46B5
:104130005DF8047B704700BF80B483B000AF786047
:104140007B689B6823F001027B689A600023184615
:104150000C37BD465DF8047B704700BF80B582B068
:1041600000AF78600B46FB707B68DB6823F0C042D1
:104170007B68DA60FB78012B06D17B68DB6843F053
:1041800000527B68DA6008E0FB78002B05D17B6881
:10419000DB6843F080427B68DA60322003F0EAFC9F
:1041A000002318460837BD4680BD00BF84B080B5E7
:1041B00084B000AF786007F11C0080E80E00002397
:1041C000FB607B689B6B43F400227B689A633B6CCB
:1041D000002B05D17B689B6B43F400127B689A63CC
:1041E0007B6803F560631A46002313607B6803F560
:1041F00000631A467B6803F500631B6813603B6B22
:10420000012B0CD17B6A002B04D17868002100F0CF
:1042100041F908E07868012100F03CF903E0786892
:10422000032100F037F97868102100F0EBF8786886
:1042300000F00EF97B6803F500631A460023136152
:104240007B6803F500631A46002353617B6803F51E
:1042500000631A464FF0FF3393617B6803F50063F8
:104260001A460023D3610023FB6031E0FB685A014A
:104270007B68134403F510631B68002B0ADAFB68A4
:104280005A017B68134403F510631A464FF09043BC
:10429000136008E0FB685A017B68134403F5106360
:1042A0001A4600231360FB685A017B68134403F528
:1042B00010631A4600231361FB685A017B6813449C
:1042C00003F510631A46FF239360FB680133FB601C
:1042D000FA69FB689A42C9D80023FB6031E0FB68A9
:1042E0005A017B68134403F530631B68002B0ADA1C
:1042F000FB685A017B68134403F530631A464FF09C
:104300009043136008E0FB685A017B68134403F58F
:1043100030631A4600231360FB685A017B6813441C
:1043200003F530631A4600231361FB685A017B686A
:10433000134403F530631A46FF239360FB6801338F
:10434000FB60FA69FB689A42C9D87B6803F5006391
:104350001A467B6803F500631B6923F480731361BD
:10436000BB6A012B17D17B6803F500631A46234B08
:1043700013637B6803F500631A467B6803F50063EB
:104380001B6B43F4803343F0030313637B6803F533
:1043900000631B6BFB607B6800229A617B686FF097
:1043A00080425A61BB6A002B05D17B689B6943F050
:1043B00010027B689A617B689A69114B13437A6893
:1043C00093617B6B002B05D07B689B6943F00802EF
:1043D0007B689A613B6C012B07D17B689B6943F03A
:1043E000804343F004037A68936100231846103732
:1043F000BD46BDE8804004B0704700BF00018000AA
:1044000000383C8080B485B000AF7860396000230C
:10441000FB603B689B0143F020027B681A61FB68EC
:104420000133FB60FB68094A934201D9032306E08C
:104430007B681B6903F02003002BF0D10023184692
:104440001437BD465DF8047B704700BF400D030084
:1044500080B485B000AF78600023FB607B681022D9
:104460001A61FB680133FB60FB68094A934201D97A
:10447000032306E07B681B6903F01003002BF0D1D7
:10448000002318461437BD465DF8047B704700BF13
:10449000400D030080B483B000AF78600B46FB7022
:1044A0007B6803F5006319467B6803F500631A68AF
:1044B000FB7813430B60002318460C37BD465DF8AC
:1044C000047B704780B485B000AF78600023FB7335
:1044D0007B6803F500639B6803F00603002B02D1A1
:1044E0000023FB731CE07B6803F500639B6803F00B
:1044F0000603022B07D07B6803F500639B6803F07B
:104500000603062B02D10323FB7309E07B6803F546
:1045100000639B6803F00603042B01D10223FB73A5
:10452000FB7B18461437BD465DF8047B704700BF1F
:1045300080B483B000AF786039603B685B78012B52
:104540003ED17B6803F5006319467B6803F5006381
:10455000DA693B681B781846012383409BB21343FA
:10456000CB613B681B785A017B68134403F51063E9
:104570001B6803F40043002B5CD13B681B785A0195
:104580007B68134403F5106318463B681B785A0197
:104590007B68134403F510631A683B689B68C3F398
:1045A0000A033968C97889040B4339680978890591
:1045B0000B43134343F0805343F40043036039E05B
:1045C0007B6803F5006319467B6803F50063DB69CC
:1045D0003A68127810460122824012041343CB61DC
:1045E0003B681B785A017B68134403F530631B68F2
:1045F00003F40043002B1DD13B681B785A017B68F4
:10460000134403F5306318463B681B785A017B68F6
:10461000134403F530631A683B689B68C3F30A03CD
:104620003968C97889040B43134343F0805343F43A
:1046300000430360002318460C37BD465DF8047B39
:10464000704700BF80B483B000AF786039603B68CA
:104650005B78012B35D17B6803F5006319467B68D5
:1046600003F50063DA6B3B681B781846012383402F
:104670009BB2DB431340CB637B6803F500631946B1
:104680007B6803F50063DA693B681B7818460123F1
:1046900083409BB2DB431340CB613B681B785A01DC
:1046A0007B68134403F5106319463B681B785A0175
:1046B0007B68134403F510631B6823F400430B600D
:1046C00034E07B6803F5006319467B6803F50063FB
:1046D000DA6B3B681B781846012383401B04DB43DD
:1046E0001340CB637B6803F5006319467B6803F5D1
:1046F0000063DA693B681B781846012383401B047A
:10470000DB431340CB613B681B785A017B68134441
:1047100003F5306319463B681B785A017B681344E4
:1047200003F530631B6823F400430B600023184635
:104730000C37BD465DF8047B704700BF90B589B06B
:1047400002AFF860B9601346FB710023FB82BB68BF
:104750005B78012B40F04681BB685B69002B3BD145
:10476000BB681B785A01FB68134403F510631946B4
:10477000BB681B785A01FB68134403F510631B697F
:1047800023F0FF5323F4C0130B61BB681B785A015D
:10479000FB68134403F510631946BB681B785A0184
:1047A000FB68134403F510631B6943F400230B619A
:1047B000BB681B785A01FB68134403F51063194664
:1047C000BB681B785A01FB68134403F510631B692F
:1047D000DB0CDB040B6186E0BB681B785A01FB68CD
:1047E000134403F510631946BB681B785A01FB6834
:1047F000134403F510631B69DB0CDB040B61BB681E
:104800001B785A01FB68134403F510631946BB6813
:104810001B785A01FB68134403F510631B6923F0EE
:10482000FF5323F4C0130B61BB681B785A01FB686C
:10483000134403F510631846BB681B785A01FB68E4
:10484000134403F510631A69BB685969BB689B6818
:104850000B44591EBB689B68B1FBF3F3D9048C4B26
:104860000B4013430361BB681B785A01FB68134478
:1048700003F510631946BB681B785A01FB681344A3
:1048800003F510631A69BB685B69C3F31203134332
:104890000B61BB68DB78012B25D1BB681B785A0103
:1048A000FB68134403F510631946BB681B785A0173
:1048B000FB68134403F510631B6923F0C0430B61CD
:1048C000BB681B785A01FB68134403F51063194653
:1048D000BB681B785A01FB68134403F510631B691E
:1048E00043F000530B61FB79012B0BD1BB681B78A4
:1048F0005A01FB68134403F510631A46BB681B6931
:10490000536116E0BB68DB78012B12D0BB685B6992
:10491000002B0ED0FB6803F500631946FB6803F516
:1049200000635B6BBA681278104601228240134321
:104930004B63BB68DB78012B2ED1FB6803F500636A
:104940009B6803F48073002B13D1BB681B785A015A
:10495000FB68134403F510631946BB681B785A01C2
:10496000FB68134403F510631B6843F000530B60AE
:1049700012E0BB681B785A01FB68134403F510630F
:104980001946BB681B785A01FB68134403F5106392
:104990001B6843F080530B60BB681B785A01FB68AF
:1049A000134403F510631946BB681B785A01FB6872
:1049B000134403F510631B6843F004430B60BB68AA
:1049C000DB78012B40F0F580BB68D968BB681A78AA
:1049D000BB685B699CB2FB790093F868234600F0E2
:1049E0004DFAE6E0BB681B785A01FB68134403F5F7
:1049F00030631946BB681B785A01FB68134403F502
:104A000030631B69DB0CDB040B61BB681B785A014C
:104A1000FB68134403F530631946BB681B785A01E1
:104A2000FB68134403F530631B6923F0FF5323F441
:104A3000C0130B61BB685B69002B2BD1BB681B7873
:104A40005A01FB68134403F530631946BB681B78B1
:104A50005A01FB68134403F530631A69BB689B680D
:104A6000C3F3120313430B61BB681B785A01FB6845
:104A7000134403F530631946BB681B785A01FB6881
:104A8000134403F530631B6943F400230B613CE0DE
:104A90000000F81FBB685A69BB689B6813445A1E24
:104AA000BB689B68B2FBF3F3FB82BB681B785A01BF
:104AB000FB68134403F530631946BB681B785A0141
:104AC000FB68134403F530631A69FB8ADB0418465C
:104AD0003A4B034013430B61BB681B785A01FB68D8
:104AE000134403F530631846BB681B785A01FB6812
:104AF000134403F530631A69BB689B68F98A01FBAC
:104B000003F3C3F3120313430361FB79012B0AD1AF
:104B1000BB681B785A01FB68134403F530631A46DF
:104B2000BB68DB685361BB68DB78012B2ED1FB6867
:104B300003F500639B6803F48073002B13D1BB68FB
:104B40001B785A01FB68134403F530631946BB68B0
:104B50001B785A01FB68134403F530631B6843F06C
:104B600000530B6012E0BB681B785A01FB681344CA
:104B700003F530631946BB681B785A01FB68134480
:104B800003F530631B6843F080530B60BB681B78F0
:104B90005A01FB68134403F530631946BB681B7860
:104BA0005A01FB68134403F530631B6843F0044368
:104BB0000B60002318461C37BD4690BD0000F81F4F
:104BC00080B485B000AFF860B9601346FB71BB6874
:104BD0005B78012B40F0D180BB685B69002B3BD137
:104BE000BB681B785A01FB68134403F51063194630
:104BF000BB681B785A01FB68134403F510631B69FB
:104C000023F0FF5323F4C0130B61BB681B785A01D8
:104C1000FB68134403F510631946BB681B785A01FF
:104C2000FB68134403F510631B6943F400230B6115
:104C3000BB681B785A01FB68134403F510631946DF
:104C4000BB681B785A01FB68134403F510631B69AA
:104C5000DB0CDB040B615AE0BB681B785A01FB6874
:104C6000134403F510631946BB681B785A01FB68AF
:104C7000134403F510631B69DB0CDB040B61BB6899
:104C80001B785A01FB68134403F510631946BB688F
:104C90001B785A01FB68134403F510631B6923F06A
:104CA000FF5323F4C0130B61BB685A69BB689B6850
:104CB0009A4203D9BB689A68BB685A61BB681B7883
:104CC0005A01FB68134403F510631946BB681B784F
:104CD0005A01FB68134403F510631B6943F4002376
:104CE0000B61BB681B785A01FB68134403F5106322
:104CF0001946BB681B785A01FB68134403F510631F
:104D00001A69BB685B69C3F3120313430B61FB7938
:104D1000012B0BD1BB681B785A01FB68134403F5C8
:104D200010631A46BB681B69536112E0BB685B697C
:104D3000002B0ED0FB6803F500631946FB6803F5F2
:104D400000635B6BBA6812781046012282401343FD
:104D50004B63BB681B785A01FB68134403F510636F
:104D60001946BB681B785A01FB68134403F51063AE
:104D70001B6843F004430B6079E0BB681B785A0161
:104D8000FB68134403F530631946BB681B785A016E
:104D9000FB68134403F530631B69DB0CDB040B6118
:104DA000BB681B785A01FB68134403F5306319464E
:104DB000BB681B785A01FB68134403F530631B6919
:104DC00023F0FF5323F4C0130B61BB685B69002B16
:104DD00003D0BB689A68BB685A61BB681B785A01EC
:104DE000FB68134403F530631946BB681B785A010E
:104DF000FB68134403F530631B6943F400230B6124
:104E0000BB681B785A01FB68134403F530631946ED
:104E1000BB681B785A01FB68134403F530631A69B9
:104E2000BB689B68C3F3120313430B61FB79012B2F
:104E30000AD1BB681B785A01FB68134403F5306341
:104E40001A46BB68DB685361BB681B785A01FB6874
:104E5000134403F530631946BB681B785A01FB689D
:104E6000134403F530631B6843F004430B600023D5
:104E700018461437BD465DF8047B704780B487B090
:104E800000AFF860B96011461A460B46FB71134635
:104E9000BB8000233B6100237B6197F82030002B0F
:104EA0001DD1BB880333002B00DA03339B103B6119
:104EB00000237B610FE0FB791A03FB68134403F5C1
:104EC00080531A46BB681B6813607B6901337B61A2
:104ED000BB680433BB607A693B699A42EBD3002319
:104EE00018461C37BD465DF8047B704780B487B018
:104EF00000AFF860B9601346FB8000237B61FB883C
:104F00000333002B00DA03339B103B6100237B61EA
:104F10000BE0FB6803F580531A68BB681A607B6975
:104F200001337B61BB680433BB607A693B699A4299
:104F3000EFD3BB6818461C37BD465DF8047B70474D
:104F400080B483B000AF786039603B685B78012B38
:104F500030D13B681B785A017B68134403F510631A
:104F60001B68002B12DB3B681B785A017B681344DB
:104F700003F5106319463B681B785A017B6813449C
:104F800003F510631B6823F080430B603B681B78BC
:104F90005A017B68134403F5106319463B681B787C
:104FA0005A017B68134403F510631B6843F4001334
:104FB0000B602FE03B681B785A017B68134403F5B4
:104FC00030631B68002B12DB3B681B785A017B683F
:104FD000134403F5306319463B681B785A017B681C
:104FE000134403F530631B6823F080430B603B6878
:104FF0001B785A017B68134403F5306319463B68FC
:105000001B785A017B68134403F530631B6843F433
:1050100000130B60002318460C37BD465DF8047B77
:10502000704700BF80B483B000AF786039603B68E0
:105030005B78012B2ED13B681B785A017B681344A7
:1050400003F5106319463B681B785A017B681344CB
:1050500003F510631B6823F400130B603B68DB78D7
:10506000032B03D03B68DB78022B41D13B681B78D4
:105070005A017B68134403F5106319463B681B789B
:105080005A017B68134403F510631B6843F0805397
:105090000B602DE03B681B785A017B68134403F5D5
:1050A000306319463B681B785A017B68134403F54B
:1050B00030631B6823F400130B603B68DB78032B21
:1050C00003D03B68DB78022B12D13B681B785A0176
:1050D0007B68134403F5306319463B681B785A011B
:1050E0007B68134403F530631B6843F080530B6007
:1050F000002318460C37BD465DF8047B704700BF9F
:1051000080B584B000AF78600023FB6014E0FB68DA
:105110005A017B68134403F510631A46FF2393601A
:10512000FB685A017B68134403F530631A46FF237A
:105130009360FB680133FB60FB680E2BE7D97B684B
:1051400003F500631A464FF0FF3393617B6803F564
:1051500000631A46002313617B6803F500631A4657
:10516000002353617B6803F500631A460023D36173
:105170007868FFF76DF978681021FFF743F900238D
:1051800018461037BD4680BD80B483B000AF78604C
:105190000B46FB707B6803F500631A467B6803F5DA
:1051A00000631B6823F4FE6313607B6803F50063F0
:1051B00019467B6803F500631A68FB781B0103F44A
:1051C000FE6313430B60002318460C37BD465DF8A1
:1051D000047B704780B582B000AF78607B6803F5D0
:1051E00000631A467B6803F500635B6823F00203E3
:1051F0005360032002F0BEFC002318460837BD466A
:1052000080BD00BF80B582B000AF78607B6803F5D9
:1052100000631A467B6803F500635B6843F0020392
:105220005360032002F0A6FC002318460837BD4651
:1052300080BD00BF80B485B000AF78600023FB6004
:105240007B685B69FB607B689B69FA681340FB6065
:10525000FB6818461437BD465DF8047B704700BFF5
:1052600080B485B000AF78607B6803F500639B690C
:10527000FB607B6803F50063DB69FA681340FB6041
:10528000FB681B0C18461437BD465DF8047B70475D
:1052900080B485B000AF78607B6803F500639B69DC
:1052A000FB607B6803F50063DB69FA681340FB6011
:1052B000FB689BB218461437BD465DF8047B704707
:1052C00080B485B000AF78600B46FB70FB785A0164
:1052D0007B68134403F530639B68FB607B6803F5D0
:1052E00000635B69FA681340FB60FB68184614377B
:1052F000BD465DF8047B704780B487B000AF78602E
:105300000B46FB707B6803F500631B697B617B6860
:1053100003F500635B6B3B61FB783A6922FA03F3A8
:10532000DB01DBB27A6913437B61FB785A017B684E
:10533000134403F510639A687B691340FB60FB68B4
:1053400018461C37BD465DF8047B704780B483B0B7
:1053500000AF78607B685B6903F0010318460C3787
:10536000BD465DF8047B704780B483B000AF7860C1
:105370007B6803F510631A467B6803F510631B68AE
:1053800023F4FF6323F0070313607B6803F50063D6
:105390009B6803F00603042B0AD17B6803F51063B6
:1053A0001A467B6803F510631B6843F00303136020
:1053B0007B6803F500631A467B6803F500635B684E
:1053C00043F480735360002318460C37BD465DF8E4
:1053D000047B704780B485B000AFF8600B467A60FC
:1053E000FB72FB6803F530631A4600231361FB6808
:1053F00003F530631A46FB6803F530631B6943F419
:1054000000231361FB6803F530631A46FB6803F55C
:1054100030631B6943F018031361FB6803F53063C5
:105420001A46FB6803F530631B6943F0C043136100
:10543000FB7A012B0CD1FB6803F530631A467B68BD
:105440005361FB6803F530631A464FF08023136005
:10545000002318461437BD465DF8047B704700BF33
:1054600080B485B000AF78600023FB60FB68013337
:10547000FB60FB68134A934201D903231BE07B685E
:105480001B69002BF2DA0023FB607B681B6943F089
:1054900001027B681A61FB680133FB60FB68094A03
:1054A000934201D9032306E07B681B6903F00103E3
:1054B000002BF0D1002318461437BD465DF8047B5D
:1054C000704700BF400D030080B582B000AF786028
:1054D0007B68002B01D1012357E07B6893F85130A2
:1054E000DBB2002B06D17B68002283F8502078685D
:1054F000FCF786FA7B68022283F851207B681B68E0
:105500007A681268126822F040021A607B681B6891
:105510007A6851687A68926811437A68D268114350
:105520007A68126911437A68526911437A689269FC
:1055300002F4007211437A68D26911437A68126AE0
:1055400011437A68926A0A431A607B681B687A681A
:105550009269120C02F004017A68526A0A435A6096
:105560007B681B687A68D26A1A617B681B687A68F4
:105570001268D26922F40062DA617B6800225A65FF
:105580007B68012283F85120002318460837BD4666
:1055900080BD00BF80B487B000AFF860B9607A60AA
:1055A0007B8000237B61FB6893F85130DBB27B6129
:1055B0007B69012B0BD0FB685B68B3F5827F73D1ED
:1055C000FB689B68002B6FD17B69222B6CD1BB6879
:1055D000002B05D07B68002B02D07B88002B01D1EB
:1055E000012362E0FB6893F85030012B01D10223C4
:1055F0005BE0FB68012283F85020FB6893F8513090
:10560000DBB2222B03D0FB68322283F85120FB68E7
:1056100000225A65FB68284ADA64FB68BA681A6394
:10562000FB687A889A86FB687A88DA86FB68234A60
:105630009A64FB687A689A63FB687A889A87FB6841
:105640007A88DA87FB689B6AB3F5005F0FD1FB6845
:105650001B68FA681268126822F400521A60FB682C
:105660001B68FA681268126842F400521A60FB68FC
:105670001B68FA681268526842F0E0025A60FB68E0
:10568000002283F85020FB681B681B6803F040036E
:10569000002B07D1FB681B68FA681268126842F099
:1056A00040021A60002300E0022318461C37BD4662
:1056B0005DF8047B704700BF51590008FD5A00088F
:1056C00080B588B000AF78600023FB610023BB6128
:1056D00000237B617B681B689B6803F00103002B40
:1056E00014BF01230023DBB2FB617B681B685B688E
:1056F00003F04003002B14BF01230023DBB2BB6186
:105700007B681B689B6803F04003002B14BF0123D8
:105710000023DBB27B61FB69002B0AD0BB69002B45
:1057200007D07B69002B04D17B689B6C7868984715
:105730008CE07B681B689B6803F00203002B14BF9E
:1057400001230023DBB2FB617B681B685B6803F00D
:105750008003002B14BF01230023DBB2BB61FB6974
:10576000002B07D0BB69002B04D07B68DB6C78680A
:1057700098476BE07B681B685B6803F02003002B95
:1057800064D07B681B689B6803F01003002B0AD071
:105790007B685B6D43F002027B685A657B681B681F
:1057A0006FF010029A607B681B689B6803F020030F
:1057B000002B12D07B685B6D43F001027B685A6559
:1057C0007B681B689B683B617B681B687A68126812
:1057D000126822F040021A603B697B681B689B6874
:1057E00003F04003002B14D07B6893F85130DBB2F8
:1057F000122B0ED07B685B6D43F004027B685A6508
:105800007B681B68DB68FB607B681B689B68FB60D0
:10581000FB687B681B689B6803F48073002B0AD0CD
:105820007B685B6D43F008027B685A657B681B6888
:105830009B68BB60BB687B685B6D002B06D07B6898
:10584000012283F851207868FBF7D4FC2037BD464D
:1058500080BD00BF80B483B000AF78600C37BD4618
:105860005DF8047B704700BF80B483B000AF786000
:105870000C37BD465DF8047B704700BF80B584B02F
:1058800000AF7860786802210022022300F066F9F8
:105890000346002B05D07B685B6D43F020027B68DC
:1058A0005A657B681B687A681268526822F0800229
:1058B0005A607B681B685B6803F04003002B44D18F
:1058C0007B681B687A681268526822F020025A606E
:1058D000786880210122022300F040F90346002B62
:1058E00005D07B685B6D43F020027B685A657B685E
:1058F0009B68002B08D17B681B68DB68FB607B68BA
:105900001B689B68FB60FB687B685B6D002B15D197
:105910007B6893F85130DBB2322B07D17B680122D0
:1059200083F851207868FBF703FA0EE07B680122C8
:1059300083F851207868FFF78DFF06E07B6801222D
:1059400083F851207868FBF755FC1037BD4680BDC1
:1059500080B582B000AF78607B68DB68002B09D12E
:105960007B681A687B681B6B581C796808631B7816
:10597000D3600AE07B681B687A68126B1288DA6071
:105980007B681B6B9A1C7B681A637B68DB8E013B10
:105990009AB27B68DA867B68DB8E002B0FD17B683E
:1059A0009B6AB3F5005F07D17B681B687A68126851
:1059B000126842F480521A607868FFF75FFF083778
:1059C000BD4680BD80B584B000AF78607B689B6ABF
:1059D000B3F5005F40D1786801210022022300F076
:1059E000BDF80346002B05D07B685B6D43F02002B9
:1059F0007B685A657B681B68DB689BB2FB81FB890F
:105A0000786801210122022300F0A8F80346002B48
:105A100005D07B685B6D43F020027B685A657B682C
:105A20001B689B6803F01003002B15D07B685B6D2F
:105A300043F002027B685A657B681B687A681268CB
:105A4000126822F400521A607B681B687A68126838
:105A5000126842F400521A607B681B687A68126808
:105A6000526822F040025A607B681B685B6803F052
:105A70008003002B3FD17B681B687A6812685268EC
:105A800022F020025A607B685B68B3F5827F11D1F7
:105A90007B689B68B3F5004F04D07B689B68B3F5C7
:105AA000806F07D17B681B687A681268126822F0E1
:105AB00040021A607B685B6D002B15D17B6893F800
:105AC0005130DBB2322B07D17B68012283F85120A1
:105AD0007868FBF72DF90EE07B68012283F85120EE
:105AE0007868FFF7C1FE06E07B68012283F8512049
:105AF0007868FBF77FFB1037BD4680BD80B582B06C
:105B000000AF78607B68DB68002B0AD17B689B6BF9
:105B1000591C7A6891637A681268D268D2B21A7096
:105B20000BE07B689B6B7A681268D26892B21A802D
:105B30007B689B6B9A1C7B689A637B68DB8F013B5D
:105B40009AB27B68DA877B68DB8F002B02D178689A
:105B5000FFF738FF0837BD4680BD00BF80B586B06F
:105B600000AFF860B9603B601346FB7100237B61B6
:105B700001F0F4FF7861FB79002B47D13DE03B68F1
:105B8000B3F1FF3F39D03B68002B07D001F0E6FFAF
:105B900002467B69D21A3B689A422ED9FB681B6881
:105BA000FA681268526822F0E0025A60FB681B68CB
:105BB000FA681268126822F040021A60FB689B6A59
:105BC000B3F5005F0FD1FB681B68FA6812681268B2
:105BD00022F400521A60FB681B68FA6812681268A7
:105BE00042F400521A60FB68012283F85120FB68DE
:105BF000002283F85020032350E0FB681B689A685A
:105C0000BB681A40BB689A42B9D146E03DE03B68A8
:105C1000B3F1FF3F39D03B68002B07D001F09EFF66
:105C200002467B69D21A3B689A422ED9FB681B68F0
:105C3000FA681268526822F0E0025A60FB681B683A
:105C4000FA681268126822F040021A60FB689B6AC8
:105C5000B3F5005F0FD1FB681B68FA681268126821
:105C600022F400521A60FB681B68FA681268126816
:105C700042F400521A60FB68012283F85120FB684D
:105C8000002283F85020032308E0FB681B689A6811
:105C9000BB681A40BB689A42B9D00023184618372F
:105CA000BD4680BD80B594B000AF78600023FB6432
:105CB0007B681B6803F00103002B47D09D4B9B685A
:105CC00003F00C03042B0BD09A4B9B6803F00C03DE
:105CD000082B07D1974B5B6803F48003002B01D09E
:105CE0000123BBE1944B00221A7001F037FFF864E6
:105CF00009E001F033FF0246FB6CD31AB3F5FA7FDB
:105D000001D90323AAE18B4B1B6803F40033002B5A
:105D1000EFD1894A7B685B68DBB213707B685B6894
:105D2000002B13D001F01AFFF86409E001F016FF10
:105D30000246FB6CD31AB3F5FA7F01D903238DE138
:105D40007C4B1B6803F40033002BEFD07B681B688F
:105D500003F00203002B61D0764B9B6803F00C0329
:105D6000002B0BD0734B9B6803F00C03082B0CD15A
:105D7000704B5B6803F48003002B06D17B68DB6803
:105D8000012B01D0012369E130E07B68DB68002B47
:105D900016D06A4B01221A6001F0E0FEF86408E0B8
:105DA00001F0DCFE0246FB6CD31A642B01D90323FD
:105DB00054E1604B1B6803F00203002BF0D015E0A8
:105DC0005E4B00221A6001F0C9FEF86408E001F0A1
:105DD000C5FE0246FB6CD31A642B01D903233DE1B7
:105DE000544B1B6803F00203002BF0D15148514B78
:105DF0001B6823F0F8027B681B69F821B964B96C51
:105E000091FAA1F17964796C3964396CB1FA81F154
:105E1000F963F96BC9B28B40134303607B681B685D
:105E200003F00803002B30D07B685B69002B16D091
:105E3000434B01221A6001F091FEF86408E001F082
:105E40008DFE0246FB6CD31A642B01D9032305E1B6
:105E5000384B5B6F03F00203002BF0D015E0384B9A
:105E600000221A6001F07AFEF86408E001F076FE84
:105E70000246FB6CD31A642B01D90323EEE02D4BB1
:105E80005B6F03F00203002BF0D17B681B6803F00B
:105E90000403002B60D0274A264B1B6C43F0805331
:105EA0001364284A274B1B6843F48073136001F086
:105EB00055FEF86408E001F051FE0246FB6CD31A6F
:105EC000642B01D90323C9E01E4B1B6803F48073C4
:105ED000002BF0D01C4B00221A7001F03FFEF8643A
:105EE0000AE001F03BFE0246FB6CD31A41F2883215
:105EF000934201D90323B1E00E4B1B6F03F0020361
:105F0000002BEED1104A7B689B68DBB213707B6874
:105F10009B68002B20D001F021FEF86416E001F010
:105F20001DFE0246FB6CD31A41F2883293420DD912
:105F3000032393E000380240023802400000474249
:105F4000800E47420070004070380240454B1B6F86
:105F500003F00203002BE2D07B689B69002B7CD00E
:105F6000404B9B6803F00C03082B74D03E4B00227F
:105F70001A6001F0F3FDF86408E001F0EFFD02465D
:105F8000FB6CD31A642B01D9032367E0354B1B68E4
:105F900003F00073002BF0D17B689B69022B5CD16E
:105FA00030487B681A6A7B685B6A47F6C071B963E0
:105FB000B96B91FAA1F17963796B3963396BB1FAF5
:105FC00081F1F962F96AC9B28B401A437B689B6A16
:105FD0005B08013B4FF44031B962B96A91FAA1F113
:105FE0007962796A3962396AB1FA81F1F961F969DC
:105FF000C9B28B401A437B68DB691A437B68DB6A52
:106000004FF07061B961B96991FAA1F1796179696B
:1060100039613969B1FA81F1F960F968C9B28B4027
:10602000134343F0005343600F4B01221A6001F009
:1060300095FDF86408E001F091FD0246FB6CD31A6F
:10604000642B01D9032309E0064B1B6803F000739E
:10605000002BF0D001E0012300E000231846503768
:10606000BD4680BD003802406000474280B584B024
:1060700000AF786039600023FB60A64B1B6803F01B
:106080000F023B689A4280F09080A24B3A68D2B2ED
:106090001A70A04B1B6803F00F023B689A4201D0B4
:1060A000012333E17B681B6803F00203002B08D057
:1060B0009949994B9B6823F0F0027B689B681343D6
:1060C0008B607B681B6803F00103002B00F0FB80F2
:1060D0007B685B68012B07D18F4B1B6803F400338F
:1060E000002B15D1012311E17B685B68022B07D1DE
:1060F000894B1B6803F00073002B09D1012305E1D4
:10610000854B1B6803F00203002B01D10123FDE046
:106110008149814B9B6823F003027B685B681343D2
:106120008B6001F01BFDF8607B685B68012B12D16E
:106130000AE001F013FD0246FB68D31A41F28832EF
:10614000934201D90323E1E0734B9B6803F00C03F6
:10615000042BEED1B7E07B685B68022B12D10AE01A
:1061600001F0FCFC0246FB68D31A41F288329342EC
:1061700001D90323CAE0684B9B6803F00C03082B8A
:10618000EED1A0E00AE001F0E9FC0246FB68D31A78
:1061900041F28832934201D90323B7E05E4B9B68FA
:1061A00003F00C03002BEED18DE07B681B6803F03D
:1061B0000203002B08D05849574B9B6823F0F0028C
:1061C0007B689B6813438B607B681B6803F001034B
:1061D000002B6BD07B685B68012B07D14E4B1B6893
:1061E00003F40033002B15D101238FE07B685B683B
:1061F000022B07D1484B1B6803F00073002B09D119
:10620000012383E0444B1B6803F00203002B01D100
:1062100001237BE04049404B9B6823F003027B68ED
:106220005B6813438B6001F099FCF8607B685B68E6
:10623000012B12D10AE001F091FC0246FB68D31A4F
:1062400041F28832934201D903235FE0324B9B68CD
:1062500003F00C03042BEED128E07B685B68022B73
:1062600012D10AE001F07AFC0246FB68D31A41F22F
:106270008832934201D9032348E0274B9B6803F0FF
:106280000C03082BEED111E00AE001F067FC024696
:10629000FB68D31A41F28832934201D9032335E0D7
:1062A0001D4B9B6803F00C03002BEED1194B3A6891
:1062B000D2B21A70174B1B6803F00F023B689A4268
:1062C00001D0012322E07B681B6803F00403002B4C
:1062D00008D01149104B9B6823F4E0527B68DB68BF
:1062E00013438B607B681B6803F00803002B09D005
:1062F0000949094B9B6823F460427B681B69DB00FA
:1063000013438B60002001F005FC00231846103772
:10631000BD4680BD003C02400038024080B491B0D0
:1063200000AF00237B630023FB6300233B63002358
:10633000BB633D4B9B6803F00C03042B06D0082B7A
:1063400007D0002B66D1394BBB6366E0384BBB638B
:1063500063E0354B5B6803F03F037B63324B5B6864
:1063600003F48003002B1CD0314A7B6BB2FBF3F2A9
:106370002D4B596847F6C0730B4047F6C071F96260
:10638000F96A91FAA1F1B962B96A7962796AB1FAE6
:1063900081F13962396AC9B2CB4003FB02F3FB6376
:1063A0001BE0224A7B6BB2FBF3F21F4B596847F6A6
:1063B000C0730B4047F6C071F961F96991FAA1F118
:1063C000B961B96979617969B1FA81F1396139697C
:1063D000C9B2CB4003FB02F3FB63134B5B6803F4CE
:1063E00040334FF44032FA60FA6892FAA2F2BA608F
:1063F000BA687A607A68B2FA82F23A603A68D2B2DF
:10640000D34001335B003B63FA6B3B6BB2FBF3F3AE
:10641000BB6302E0054BBB6300BFBB6B1846443750
:10642000BD465DF8047B7047003802400024F4004C
:1064300000127A0080B584B000AFFFF76FFF01460D
:106440000F4B9B6803F0F003F022FA60FA6892FAAF
:10645000A2F2BA60BA687A607A68B2FA82F23A60F6
:106460003A68D2B2D340074AD35C21FA03F3064A12
:106470001360054B1B6818461037BD4680BD00BF32
:10648000003802406C7E0008DC00002080B485B03B
:1064900000AF78600B46FB7013463B800023FB7314
:1064A0000023BB607B681B685B6ABB60FB78002BCA
:1064B00008D17B681B683A8812041146BA680A43FF
:1064C0009A6229E07B681B689B6A1B0CBA681344BC
:1064D000BB600023FB730DE07B681A68FB7B4033D5
:1064E0009B0013445B681B0CBA681344BB60FB7BC6
:1064F0000133FB73FA7BFB78013B9A42ECDB7B6850
:106500001968FB78013B3A8812041046BA680243C6
:1065100040339B000B445A60002318461437BD4695
:106520005DF8047B704700BF80B483B000AF786033
:106530000B467B807B681B687A885A62002318466A
:106540000C37BD465DF8047B704700BFF0B58FB0D7
:106550000AAF78600023FB607B68002B01D1012328
:10656000F7E07B68032283F87D237868F9F794FECF
:106570007B681B681846FDF7DFFD7B68D3F800E0F9
:106580007E686D4606F110040FCC0FC50FCC0FC509
:1065900023682B60331D0ECB7046FDF769FD7B68C9
:1065A0001B6818460021FDF7D9FD0023FB604CE075
:1065B0007968FA681346DB009B1A9B000B44303362
:1065C00001225A71FB68D8B27968FA681346DB0079
:1065D0009B1A9B000B44303302461A71FB6898B239
:1065E0007968FA681346DB009B1A9B000B44303332
:1065F00002465A817968FA681346DB009B1A9B00B1
:106600000B4430330022DA717968FA681346DB00F4
:106610009B1A9B000B44383300225A607968FA6851
:106620001346DB009B1A9B000B44383300229A6010
:106630007968FA681346DB009B1A9B000B444033D1
:1066400000229A60FB680133FB60FB680E2BAFD918
:106650000023FB605AE07968FA681346DB009B1A56
:106660009B000B4403F5EC7300225A70FB68D8B210
:106670007968FA681346DB009B1A9B000B4403F50C
:10668000EC7302461A70FB6898B27968FA68134690
:10669000DB009B1A9B000B44303302465A81796819
:1066A000FA681346DB009B1A9B000B4403F5EC735E
:1066B0000022DA707968FA681346DB009B1A9B00A7
:1066C0000B4403F5F07300221A607968FA681346E8
:1066D000DB009B1A9B000B4403F5F07300225A6009
:1066E0007968FA681346DB009B1A9B000B4403F59C
:1066F000F47300225A607B681A68FB6840339B0081
:10670000134400225A60FB680133FB60FB680E2BC8
:10671000A1D97B68D3F800E07E686D4606F11004CD
:106720000FCC0FC50FCC0FC523682B60331D0ECBCC
:106730007046FDF73BFD7B68012283F87D237B6873
:10674000002283F87C237B681B681846FEF75AFDFD
:10675000002318461437BD46F0BD00BF80B582B097
:1067600000AF78607B6893F87C33012B01D1022362
:1067700012E07B68012283F87C237B681B68184643
:10678000FEF728FD7B681B681846FDF7C3FC7B6895
:10679000002283F87C23002318460837BD4680BDBD
:1067A00080B582B000AF78607B6893F87C33012BB2
:1067B00001D1022317E07B68012283F87C237B68E8
:1067C0001B681846FDF7B8FC7B681B681846FEF787
:1067D00097FC7B681B681846FEF714FD7B68002257
:1067E00083F87C23002318460837BD4680BD00BFD0
:1067F00080B58AB000AF78607B681B68BB610023FE
:106800007B6200233B6200237B610023FB6100234A
:106810003B610023FB607B681B681846FEF796FD12
:106820000346002B40F092837B681B681846FEF7F6
:1068300001FD0346002B00D188E37B681B681846E6
:10684000FEF7F8FC034603F00203002B03D07B683D
:106850001B6802225A617B681B681846FEF7EAFC37
:10686000034603F40023002B00F0B3800023FB61F8
:106870007B681B681846FEF7F3FC3862A5E03B6AAC
:1068800003F00103002B00F09A807B681A68FB6913
:10689000DBB210461946FEF713FD78617B6903F001
:1068A0000103002B6CD0FB695A01BB69134403F54B
:1068B00030631A46012393607B681B69012B3CD12E
:1068C0007968FA691346DB009B1A9B000B4403F5B9
:1068D000F0731A68FB695901BB690B4403F5306317
:1068E0001B69C3F31203D11A7868FA691346DB00F7
:1068F0009B1A9B00034403F5F87319607968FA69E1
:106900001346DB009B1A9B000B4403F5F073596898
:106910007868FA691346DB009B1A9B00034403F571
:10692000F0731B6819447868FA691346DB009B1AF8
:106930009B00034403F5F0735960FB69DBB2786890
:106940001946F9F7F1FC7B681B69012B18D1FB692B
:10695000002B15D17968FA691346DB009B1A9B005E
:106960000B4403F5F4735B68002B09D17B681A684C
:106970007B6803F56073104601211A46FEF72AFD75
:106980007B6903F00803002B0BD07868F9F7BAFC99
:10699000FB695A01BB69134403F530631A460823A7
:1069A00093607B6903F01003002B08D0FB695A0148
:1069B000BB69134403F530631A4610239360FB69E7
:1069C0000133FB613B6A5B083B623B6A002B7FF44F
:1069D00056AF7B681B681846FEF72CFC034603F491
:1069E0008023002B00F0C4807B681B681846FEF7EC
:1069F0004FFC38620023FB61B6E03B6A03F0010301
:106A0000002B00F0AB807B681A68FB69DBB2104694
:106A10001946FEF771FC78617B6903F00103002BD6
:106A20005BD0FB69012202FA03F33B61BB6903F50A
:106A300000631946BB6903F500635A6B3B69DB438E
:106A400013404B63FB695A01BB69134403F51063A0
:106A50001A46012393607B681B69012B1BD179685F
:106A6000FA691346DB009B1A9B000B443833996884
:106A70007868FA691346DB009B1A9B00034438339D
:106A80005B6819447868FA691346DB009B1A9B001F
:106A9000034438339960FB69DBB278681946F9F72B
:106AA0005FFC7B681B69012B17D1FB69002B14D19C
:106AB0007968FA691346DB009B1A9B000B4440334C
:106AC0009B68002B09D17B681A687B6803F56073AB
:106AD000104601211A46FEF77DFC7B6903F008038E
:106AE000002B08D0FB695A01BB69134403F51063FE
:106AF0001A46082393607B6903F01003002B08D02B
:106B0000FB695A01BB69134403F510631A4610234D
:106B100093607B6903F04003002B08D0FB695A01A6
:106B2000BB69134403F510631A46402393607B69E5
:106B300003F00203002B08D0FB695A01BB69134420
:106B400003F510631A46022393607B6903F0800308
:106B5000002B03D07868F96900F076FCFB690133FB
:106B6000FB613B6A5B083B623B6A002B7FF445AFED
:106B70007B681B681846FEF75DFB0346002B12DAA4
:106B8000BB6903F500631A46BB6903F500635B68E4
:106B900023F0010353607868F9F74CFC7B681B68AD
:106BA0004FF000425A617B681B681846FEF742FBB3
:106BB000034603F40063002B0FD0BB6903F50063A9
:106BC0009B6803F00103002B02D07868F9F718FCEA
:106BD0007B681B684FF400625A617B681B6818462B
:106BE000FEF728FB034603F48053002B00F090804F
:106BF000BB6903F500631A46BB6903F500635B6874
:106C000023F0010353607B681B6818460021FDF7E1
:106C1000F9FB00237B6214E07B6A5A01BB691344D1
:106C200003F510631A46FF2393607B6A5A01BB6920
:106C3000134403F530631A46FF2393607B6A0133E4
:106C40007B627B685A687B6A9A42E5D8BB6903F528
:106C500000631A464FF0FF339361BB6903F500638D
:106C60001A46BB6903F50063DB6943F00113D36186
:106C70007B68DB6A002B18D0BB6903F500631A46FA
:106C8000BB6903F50063D3F8843043F00B03C2F80B
:106C90008430BB6903F500631A46BB6903F50063E2
:106CA0005B6C43F00B03536415E0BB6903F50063B1
:106CB0001A46BB6903F500635B6943F00B0353613C
:106CC000BB6903F500631A46BB6903F500631B69E2
:106CD00043F00B031361BB6903F500631A46BB69FC
:106CE00003F500631B6823F4FE6313607B68196877
:106CF0007B681B69DAB27B6803F56073084611464E
:106D00001A46FEF767FB7B681B684FF480525A6196
:106D10007B681B681846FEF78DFA034603F40053A0
:106D2000002B3AD07B681B681846FEF71DFB7B687A
:106D30001B687A681268D26822F47052DA607B6845
:106D40001B681846FDF7BEFB0346002B0FD17B687E
:106D50000022DA607B684FF400725A617B681B681E
:106D60007A681268D26842F41052DA600DE07B68EB
:106D70000322DA607B6840225A617B681B687A686C
:106D80001268D26842F4A052DA607868F9F710FB12
:106D90007B681B684FF400525A617B681B68184679
:106DA000FEF748FA034603F01003002B63D07B681C
:106DB0001B687A681268926922F010029A61BB69B6
:106DC0001B6AFB60FB6803F00F021346DB009B1A93
:106DD0009B0003F5EC737A681344BB60FB6803F413
:106DE000F0135B0C022B26D1FA6847F6F0731340C0
:106DF000002B38D0BB68D968FA6847F6F0731340A7
:106E00001B099BB2B8691A46FEF770F8BB68DA68CE
:106E1000F96847F6F0730B401B091A44BB68DA6047
:106E2000BB689A69F96847F6F0730B401B091A446E
:106E3000BB689A6117E0FB6803F4F0135B0C062B48
:106E400011D17B6803F56073B86919460822FEF713
:106E50004DF8BB689A69F96847F6F0730B401B0957
:106E60001A44BB689A617B681B687A6812689269E9
:106E700042F010029A617B681B681846FEF7DAF947
:106E8000034603F00803002B06D07868F9F782FA6E
:106E90007B681B6808225A617B681B681846FEF7EE
:106EA000C9F9034603F48013002B0AD0FB69DBB257
:106EB00078681946F9F7EAFA7B681B684FF4801284
:106EC0005A617B681B681846FEF7B4F9034603F461
:106ED0000013002B0AD0FB69DBB278681946F9F77A
:106EE000C3FA7B681B684FF400125A617B681B6809
:106EF0001846FEF79FF9034603F08043002B07D0A6
:106F00007868F9F7D5FA7B681B684FF080425A61C0
:106F10007B681B681846FEF78DF9034603F00403EF
:106F2000002B13D07B681B685B68FB60FB6803F079
:106F30000403002B02D07868F9F7C8FA7B681B6855
:106F40007A6812685168FA680A435A602837BD4661
:106F500080BD00BF80B582B000AF78600B46FB708B
:106F60007B6893F87C33012B01D102230FE07B680F
:106F7000012283F87C237B681A68FB781046194647
:106F8000FEF702F97B68002283F87C230023184671
:106F90000837BD4680BD00BF80B584B000AF7860C3
:106FA000084611461A460346FB700B463B801346C3
:106FB000BB700023FB72FB785BB2002B0CDAFB7812
:106FC00003F07F021346DB009B1A9B0030337A6884
:106FD00013440433FB600BE0FB7803F07F0213469D
:106FE000DB009B1A9B0003F5EC737A681344FB608B
:106FF000FB7803F07F03DAB2FB681A70FB78DB09D9
:10700000DBB21A46FB685A703A88FB689A60FB68E4
:10701000BA78DA70FB685B78002B04D0FB681B78C9
:107020009AB2FB68DA80BB78022B02D1FB6800229F
:107030001A717B6893F87C33012B01D102230EE097
:107040007B68012283F87C237B681B681846F968FB
:10705000FDF76EFA7B68002283F87C23FB7A1846E2
:107060001037BD4680BD00BF80B584B000AF7860EA
:107070000B46FB70FB785BB2002B0CDAFB7803F05D
:107080007F021346DB009B1A9B0030337A6813445F
:107090000433FB600BE0FB7803F07F021346DB0058
:1070A0009B1A9B0003F5EC737A681344FB60FB7832
:1070B00003F07F03DAB2FB681A70FB78DB09DBB2FE
:1070C0001A46FB685A707B6893F87C33012B01D118
:1070D00002230EE07B68012283F87C237B681B6817
:1070E0001846F968FDF7AEFA7B68002283F87C2326
:1070F000002318461037BD4680BD00BF80B586B05E
:1071000000AFF8607A603B600B46FB72FB7A03F0DD
:107110007F021346DB009B1A9B0003F5EC73FA68B1
:1071200013447B617B697A68DA607B693A685A61EB
:107130007B6900229A617B6900225A70FB7A03F016
:107140007F03DAB27B691A70FB681B69012B02D1DD
:107150007A687B691A61FB6893F87C33012B01D153
:10716000022322E0FB68012283F87C23FB7A03F0F0
:107170007F03002B0AD1FB681A68FB681B69DBB22E
:10718000104679691A46FDF71BFD09E0FB681A688D
:10719000FB681B69DBB2104679691A46FDF7CEFA27
:1071A000FB68002283F87C23002318461837BD466D
:1071B00080BD00BF80B483B000AF78600B46FB7029
:1071C000FB7803F07F0279681346DB009B1A9B0073
:1071D0000B4403F5F8731B689BB218460C37BD4689
:1071E0005DF8047B704700BF80B586B000AFF860E3
:1071F0007A603B600B46FB72FB7A03F07F0213461A
:10720000DB009B1A9B003033FA68134404337B6124
:107210007B697A68DA607B693A685A617B69002227
:107220009A617B6901225A70FB7A03F07F03DAB21C
:107230007B691A70FB681B69012B02D17A687B6934
:107240001A61FB6893F87C33012B01D1022322E001
:10725000FB68012283F87C23FB7A03F07F03002B79
:107260000AD1FB681A68FB681B69DBB210467969B2
:107270001A46FDF7A5FC09E0FB681A68FB681B6964
:10728000DBB2104679691A46FDF758FAFB6800220E
:1072900083F87C23002318461837BD4680BD00BF05
:1072A00080B584B000AF78600B46FB70FB785BB2B2
:1072B000002B0CDAFB7803F07F021346DB009B1AED
:1072C0009B0030337A6813440433FB6009E0FA789A
:1072D0001346DB009B1A9B0003F5EC737A6813449A
:1072E000FB60FB6801229A70FB7803F07F03DAB23F
:1072F000FB681A70FB78DB09DBB21A46FB685A7030
:107300007B6893F87C33012B01D1022320E07B685A
:10731000012283F87C237B681B681846F968FDF717
:107320000FFEFB7803F07F03002B0CD17B681968FC
:107330007B681B69DAB27B6803F560730846114607
:107340001A46FEF747F87B68002283F87C23002367
:1073500018461037BD4680BD80B584B000AF786058
:107360000B46FB70FB785BB2002B0CDAFB7803F06A
:107370007F021346DB009B1A9B0030337A6813446C
:107380000433FB6009E0FA781346DB009B1A9B008C
:1073900003F5EC737A681344FB60FB6800229A7073
:1073A000FB7803F07F03DAB2FB681A70FB78DB0925
:1073B000DBB21A46FB685A707B6893F87C33012B6A
:1073C00001D102230EE07B68012283F87C237B68D5
:1073D0001B681846F968FDF725FE7B68002283F8D4
:1073E0007C23002318461037BD4680BD80B582B08F
:1073F00000AF78600B46FB707B6893F87C33012B01
:1074000001D102231BE07B68012283F87C23FB78F7
:107410005BB2002B09DA7B681A68FB7803F07F0304
:1074200010461946FCF7EEFF04E07B681B6818461F
:10743000FDF70EF87B68002283F87C2300231846B2
:107440000837BD4680BD00BF90B58BB002AF7860F5
:1074500039607B681B687B610023FB6100233B6113
:107460003A681346DB009B1A9B0030337A6813445A
:107470000433FB60FB685A69FB689B69D31AFB61A4
:10748000FA69FB689B689A4202D9FB689B68FB61BA
:10749000FB690333002B00DA03339B10BB612EE042
:1074A000FB68D9683B68DAB2FB699CB27B681B69F0
:1074B000DBB2009378692346FDF7E0FCFB68DA68ED
:1074C000FB691A44FB68DA60FB689A69FB691A4435
:1074D000FB689A61FB685A69FB689B69D31AFB6178
:1074E000FA69FB689B689A4202D9FB689B68FB615A
:1074F000FB690333002B00DA03339B10BB613B684D
:107500005A017B69134403F510639B699AB2BB6906
:107510009A4209D3FB689A69FB685B699A4203D275
:10752000FB685B69002BBBD1FB69002B13DC3B685C
:10753000012202FA03F33B617B6903F500631946FC
:107540007B6903F500635A6B3B69DB4313404B6374
:107550007868F8F7C9FF002318462437BD4690BD68
:1075600080B487B000AF786039600023FB600023EF
:10757000BB6000233B6100237B6165E17B690122E5
:1075800002FA03F3FB603B681A68FB681340BB60B8
:10759000BA68FB689A4240F054813B685B68022BF2
:1075A00003D03B685B68122B22D17B69DA087B68C9
:1075B000083253F822303B617B6903F007039B00DC
:1075C0001A460F239340DB433A6913403B613B6803
:1075D0001B697A6902F00702920093403A691343EB
:1075E0003B617B69DA087B680832396943F822100D
:1075F0007B681B683B617B695B001A4603239340F1
:10760000DB433A6913403B613B685B6803F003036B
:107610007A69520093403A6913433B617B683A6947
:107620001A603B685B68012B0BD03B685B68022BE0
:1076300007D03B685B68112B03D03B685B68122B5B
:107640002FD17B689B683B617B695B001A460323F3
:107650009340DB433A6913403B613B68DB687A69DE
:10766000520093403A6913433B617B683A699A60E0
:107670007B685B683B617B69012202FA03F3DB43B1
:107680003A6913403B613B685B6803F010031A09D9
:107690007B6902FA03F33A6913433B617B683A69F9
:1076A0005A607B68DB683B617B695B001A46032399
:1076B0009340DB433A6913403B613B689B687A69BE
:1076C000520093403A6913433B617B683A69DA6040
:1076D0003B685B6803F08053002B00F0B2805F4A88
:1076E0005E4B5B6C43F4804353645D4A7B699B084B
:1076F000023352F823303B617B6903F003039B00A4
:107700001A460F239340DB433A6913403B617B6881
:10771000544A934231D07B68534A93422BD07B68C2
:10772000524A934225D07B68514A93421FD07B68CE
:10773000504A934219D07B684F4A934213D07B68DA
:107740004E4A93420DD07B684D4A934207D07B68E6
:107750004C4A934201D1082310E009230EE007238D
:107760000CE006230AE0052308E0042306E00323D7
:1077700004E0022302E0012300E000237A6902F022
:107780000302920093403A6913433B6134497B6999
:107790009B0802333A6941F823203B4B1B683B614D
:1077A000BB68DB433A6913403B613B685B6803F4A9
:1077B0008033002B03D03A69BB6813433B61324AE4
:1077C0003B691360304B5B683B61BB68DB433A69E4
:1077D00013403B613B685B6803F40033002B03D02C
:1077E0003A69BB6813433B61274A3B695360264BA8
:1077F0009B683B61BB68DB433A6913403B613B6874
:107800005B6803F48013002B03D03A69BB68134311
:107810003B611D4A3B6993601B4BDB683B61BB6866
:10782000DB433A6913403B613B685B6803F4001338
:10783000002B03D03A69BB6813433B61124A3B6992
:10784000D3607B6901337B617B690F2B7FF696AE3A
:107850001C37BD465DF8047B704700BF003802400E
:1078600000380140000002400004024000080240CD
:10787000000C0240001002400014024000180240B8
:10788000001C024000200240003C014080B485B052
:1078900000AF78607B6803F00703FB600C4BDB688C
:1078A000BB60BA684FF6FF031340BB60FB681A0267
:1078B000BB68134343F0BF6343F40033BB60044A27
:1078C000BB68D3601437BD465DF8047B704700BFCA
:1078D00000ED00E080B400AF044BDB6803F4E0632C
:1078E0001B0A1846BD465DF8047B704700ED00E0BA
:1078F00080B483B000AF0346FB71084997F90730A5
:107900005B09FA7902F01F02012000FA02F241F845
:1079100023200C37BD465DF8047B704700E100E092
:1079200080B483B000AF03463960FB7197F907302C
:10793000002B0BDA0D49FB7903F00F03043B3A6887
:10794000D2B21201D2B20B441A7609E0084997F973
:1079500007303A68D2B21201D2B20B4483F8002346
:107960000C37BD465DF8047B704700BF00ED00E0BA
:1079700000E100E080B489B000AFF860B9607A60DF
:10798000FB6803F00703FB61FB69C3F10703042BEA
:1079900028BF0423BB61FB690433062B02D9FB69B2
:1079A000033B00E000237B61BB69012202FA03F381
:1079B000013B1A46BB681A407B699A407B690121EA
:1079C00001FA03F3013B19467B680B401343184649
:1079D0002437BD465DF8047B704700BF80B483B098
:1079E00000AF78607B68013BB3F1807F01D3012356
:1079F0000AE0084A7B68013B5360064B00229A600C
:107A0000044B07221A60002318460C37BD465DF868
:107A1000047B704710E000E080B582B000AF786072
:107A20007868FFF733FF0837BD4680BD80B586B064
:107A300000AF0346B9607A60FB7300237B61FFF7F8
:107A400049FF78617869B9687A68FFF793FF024661
:107A500097F90F3018461146FFF762FF1837BD46F9
:107A600080BD00BF80B582B000AF0346FB7197F9BF
:107A700007301846FFF73CFF0837BD4680BD00BF02
:107A800080B582B000AF78607868FFF7A7FF034643
:107A900018460837BD4680BD80B483B000AF78601B
:107AA0007B68042B06D1094A084B1B6843F004038A
:107AB000136005E0054A054B1B6823F004031360BF
:107AC0000C37BD465DF8047B704700BF10E000E056
:107AD00080B500AF0E4A0E4B1B6843F40073136071
:107AE0000B4A0B4B1B6843F480631360084A084B36
:107AF0001B6843F4807313600320FFF78DFF0020A1
:107B000000F008F8F9F772FF0023184680BD00BFA7
:107B1000003C024080B582B000AF7860FEF78AFC7E
:107B20000246064BA3FB02239B091846FFF7A8FF5A
:107B3000002318460837BD4680BD00BFD34D6210F4
:107B400080B400AF044B1B680133034A1360BD4689
:107B50005DF8047B704700BF6401002080B400AF73
:107B6000034B1B681846BD465DF8047B704700BF99
:107B70006401002080B584B000AF78600023FB6012
:107B8000FFF7ECFFF86000BFFFF7E8FF0246FB6875
:107B9000D21A7B689A42F7D31037BD4680BD00BF2A
:107BA00080B400AF124A124B1B6843F0010313600C
:107BB0000F4B00229A600E4A0D4B1B6823F0847312
:107BC00023F4803313600A4B0A4A5A60084A084B70
:107BD0001B6823F480231360054B0022DA60064BF8
:107BE0004FF000629A60BD465DF8047B704700BFAD
:107BF000003802401030002400ED00E0DFF830D003
:107C0000002103E00B4B5B58435004310A480B4BF7
:107C100042189A42F6D30A4A02E0002342F8043B93
:107C2000084B9A42F9D3FFF7BBFFF9F77FFD704786
:107C300000C001207E7E00080000002044010020DA
:107C400048010020100E0020FEE70000024B014614
:107C5000186800F04FB800BF40010020024B0146F9
:107C6000186800F003B800BF4001002030B50029BB
:107C70003CD051F8042C0B1F1D49002AB8BF9B189B
:107C80000A680C4612B95A600B6030BD93420DD29F
:107C900019685818904201BF5A5852181A60426821
:107CA00023605A6030BD994203D80A4651680029C2
:107CB000F9D1146815199D420AD11B682344D018C4
:107CC0008842136012D10868034413604B680CE0CB
:107CD00002D90C23036030BD1C681819884201BF0B
:107CE00008684968001918605960536030BD00BFCA
:107CF0006C01002070B5CC1C24F0030408340C2C5B
:107D000038BF0C24002C064603DA0C233360002015
:107D100070BD8C42F9D3204A136810461946A1B1B0
:107D20000A68121B0ED40B2A03D90A608B188C50D8
:107D30001FE08B420BBF5A684A6802605A6018BF46
:107D40000B4616E00B464968E9E7144D2B681BB952
:107D5000304600F025F828603046214600F020F833
:107D6000421C0346D1D0C51C25F0030585420AD12B
:107D70001C6003F10B001A1D20F00700821A0AD0C4
:107D80005142995070BD3046E91A00F009F80130AF
:107D9000BBD02B46ECE770BD6C01002068010020D1
:107DA00038B5064C002305460846236000F008F865
:107DB000431C02D1236803B12B6038BD0C0E002098
:107DC000044A05491368002B08BF0B46184410608D
:107DD0001846704770010020100E0020008002023B
:107DE0001F00000053544D202020202050726F644B
:107DF000756374202020202020202020302E303158
:107E000053544D3332204D6173732053746F72613C
:107E10006765000053544D6963726F656C656374E8
:107E2000726F6E6963730000303030303030303044
:107E300030303141000000004D534320436F6E66E7
:107E4000696700004D534320496E74657266616333
:107E500065000000000000030080830000000000B7
:107E6000000000000006000000000000000000000C
:0E7E700001020304010203040607080943008F
:107E7E0089010008AD010008F9010008D1010008D0
:107E8E0021020008490200087102000812010002D6
:107E9E000000004083042A57000201020301000083
:107EAE0004030904293D0008B93D0008053E0008F9
:107EBE000000000000000000713F0008913F000824
:107ECE00000000000000000000000000B13F0008AC
:107EDE00F13F0008114000083140000851400008F1
:107EEE0009022000010104C0FA090400000208067C
:107EFE00500507058102000200070501020002007D
:107F0E0009022000010104C0320904000002080623
:107F1E0050050705810240000007050102400000E0
:107F2E0009072000010104C03209040000020806FE
:107F3E0050050705810240000007050102400000C0
:107F4E000A06000200000040010000000024F400B8
:107F5E000000000000000000000000000000000013
:107F6E000000000000000000000000000000000003
:107F7E007C7E0008000000000000000000000000F1
:107F8E0000000000000000000000000000000000E3
:107F9E0000000000000000000000000000000000D3
:107FAE0000000000000000000000000000000000C3
:047FBE00E0000020BF
:0400000508007BFD77
:00000001FF
